:020000021000EC
:10C000000000022075C301005DC301005FC3010091
:10C0100061C3010063C3010065C3010000000000AB
:10C0200000000000000000000000000067C30100E5
:10C0300069C30100000000006BC301006DC3010073
:10C040006FC301006FC30100DDEB01006FC301008E
:10C050006FC301006FC3010031EA0100FDEC010074
:10C060006FC301006FC301006FC301006FC3010004
:10C070006FC301006FC301006FC301006FC30100F4
:10C08000E9EB010035CA01006FC301006FC3010075
:10C090006FC301006FC30100C94502006FC30100F7
:10C0A0006FC301006FC301006FC301006FC30100C4
:10C0B0006FC301006FC3010000000000000000001A
:10C0C0006FC301006FC301006FC301006FC30100A4
:10C0D0002DF201006FC301006FC301006FC30100A7
:10C0E0006FC301000000000000000000000000001D
:10C0F000000000006FC30100000000006FC30100DA
:10C10000000000000000000000000000000000002F
:10C11000000000000000000000000000000000001F
:10C12000000000000000000000000000000000000F
:10C1300000000000000000000000000000000000FF
:10C1400000000000000000000000000000000000EF
:10C1500000000000000000000000000000000000DF
:10C1600000000000000000000000000000000000CF
:10C1700000000000000000000000000000000000BF
:10C1800000000000000000000000000000000000AF
:10C19000000000000000000000000000000000009F
:10C1A000000000000000000000000000000000008F
:10C1B000000000000000000000000000000000007F
:10C1C000000000000000000000000000000000006F
:10C1D000000000000000000000000000000000005F
:10C1E000000000000000000000000000000000004F
:10C1F000000000000000000000000000000000003F
:10C20000354936480A1A02D0072291438D463449EF
:10C2100034480A1A06D00722914381F30988022282
:10C2200082F3148830483149314A00F044F83148EB
:10C230003149324A00F03FF831483249324A00F081
:10C240003AF832483249334A00F035F83248334937
:10C25000334A00F030F833483349344A00F02BF8C1
:10C2600033483449344A00F026F83448344900222F
:10C2700000F02CF833483449002200F027F8334806
:10C280003349091A082902DB002202604160314A61
:10C2900090471F481F49884205D00268043003B404
:10C2A000904703BCF7E700208646EC4600200021BB
:10C2B000294A9047FEE7884207D0521A05D00378F2
:10C2C00001300B700131013AF9D17047884202D038
:10C2D00002700130FAE770470000022000F80120E8
:10C2E00000000220000002208455020020260020C9
:10C2F0003C270020D0C30100D0C3010072530200CC
:10C300008455020020260020202600200054020030
:10C3100000540200005402000054020000540200C5
:10C320000054020000540200005402008455020030
:10C33000A05602003C2700203C2700203C2700207C
:10C340009C3500209C350020A0350020A035002021
:10C35000A03D00209DC301001DFB0100FEE7FEE79C
:10C36000FEE7FEE7FEE7FEE7FEE7FEE7FEE7FEE7A5
:10C3700000F002B8FFF7FCBF0F484FF007018843F9
:10C3800085460E4880470E48016841F470010160FF
:10C39000BFF34F8FBFF36F8FFFF732BF09480A49D2
:10C3A0000A4A884207D0521A05D0037801300B7030
:10C3B0000131013AF9D170470000022021E3010068
:10C3C00088ED00E0EC5302000C260020202600201F
:10C3D00000487047943500201FB50021039001AA42
:10C3E00044F20100CDE9011100F004F805B05DF858
:10C3F00004FB000072B6094B1B68DB0700D500BECA
:10C40000BFF34F8F0649074BCA6802F4E06213433B
:10C41000CB60BFF34F8F00BFFDE700BFF0ED00E042
:10C4200000ED00E00400FA05D0E90223D1E90201A1
:10C43000994208BF90422CBF0120002070470000A5
:10C4400008B50B4800F0E1FA0A4B0B49D3E9002389
:10C450001218D1E9000143F100038B4208BF824268
:10C4600003D212F1807243F100031046194608BD51
:10C470002026002040270020B827002037B5054699
:10C480000C460A4801A901F068FA60B105704460E1
:10C4900001A9064801F08BFA18B1054800F0BAFA74
:10C4A000002003B030BD0420FBE700BFA42700201C
:10C4B0002026002038B5184B1B78044613B90025F8
:10C4C000284638BD0028FAD0037F03F0FF05002B73
:10C4D000F5D0FFF7B5FFD4E90223994208BF904297
:10C4E00014D3236903B92377D4E905309847216928
:10C4F0000029E4D0237F03F0FF05002BDFD0D4E92F
:10C500000223521843F10003C4E9022303482146E1
:10C5100001F0F8FDD4E700BF4827002004540200D2
:10C5200013B5114B1149186801900823104858227F
:10C5300001F0DEF9044698B90E4A0F4801A900F04F
:10C5400069F9044660B90C48012100F041FA012361
:10C550000A4A0948194600F0A3F9094B01221A704A
:10C56000204602B010BD00BF005402004C2700203E
:10C57000A4270020EDC5010020260020FFFF7F003A
:10C58000482700203AB103685A614A1E514251417E
:10C590001961002070470720704738B5037F0446B3
:10C5A0000D4683B98261FFF74BFF2369401941F1C2
:10C5B0000001C4E9020103B1256121460020BDE864
:10C5C0003840FFF75BBF002038BD002301460377EA
:10C5D0000120FFF753BF401A20F07F407047000052
:10C5E000014800F012BA00BF202600202DE9F04FCC
:10C5F00085B0804600F0F4F940B15A4AD2E90031E2
:10C6000013F1807341F10001C2E90031002140467D
:10C6100000F0F5F938B1544E336823B13068FFF7B4
:10C6200049FF002333600121404600F0E8F920B1C2
:10C63000FFF706FF4D4BC3E900014D484A4F4D4EF1
:10C64000DFF8389103A901F0C2F9002845D1DFF8DD
:10C650002491454EDFF828A1484601F069FD336872
:10C66000002875D07BB13368D0E90201D3E90223F9
:10C67000994208BF90422DD233681B7F1BB13168AD
:10C68000484601F03FFD484601F04CFDD0E902B3B9
:10C6900007460193FFF7D4FE019BBBEB000463EB5D
:10C6A0000105012C75F1000345DBB4F5350F40D3CE
:10C6B000FFF796FF304A02444FF49603002150469C
:10C6C00000F00EF900283ED1336813B9404600F05F
:10C6D000DFF8376005B0BDE8F08F0378012B1DD07F
:10C6E000022B09D14FF0000A304601F01BFD002853
:10C6F00034D080F81CA0F7E73BB941680B7F23B921
:10C7000001230B77304601F0FDFC03A9184801F026
:10C7100089F903A9164801F05AF996E741683B6880
:10C72000994202D100233B60EFE7304601F003FD60
:10C73000EBE7BA68C0E70021504600F056F93846EA
:10C74000FFF7B8FE01E00D28F9D00023336083E73E
:10C75000002BBFD1404600F09FF8BBE7012389F8CA
:10C760000030D2E740270020C0270020B827002053
:10C77000A427002004540200FFFFB4004827002033
:10C780002026002070B5EFF3108672B60C4A94682C
:10C7900001239CB993600B4B0B4DD3F880102940BB
:10C7A0001160C3F88050D3F8841051604FF0FF320D
:10C7B000C3F88420047006B962B670BD0370FAE74E
:10C7C000C427002000E100E0FC06FFBD084B9A688A
:10C7D00010B55AB150B9EFF3108172B6054A1C6812
:10C7E00014605C685460986001B962B610BD00BF07
:10C7F000C427002000E100E0435882B03BB1002391
:10C80000435043580193019B012002B070471846E2
:10C81000FBE70000F0B51A4B46791A4C43F8262086
:10C8200004EBC603F7001B793BBB03680A88C3F817
:10C83000082590F904508A780379002DADBF05F1E1
:10C840006041114903F00F0C01F561414FEA4212BA
:10C85000D2B2B4BF01F80C2081F800236D09012287
:10C860000A4903F01F0302FA03F341F82530E319E4
:10C8700044F836001A710020F0BD0820FCE700BF24
:10C88000D8270020D027002014ED00E000E100E0D0
:10C89000036801221A607047036801225A607047DA
:10C8A00073B501F15005AD000068ADB24FF48034AE
:10C8B0008C400026C0F80843C0F84843465101F5B3
:10C8C000A8714559019522F07F42019D40F8212031
:10C8D000C0F844430BB1C0F8044302B070BD00007F
:10C8E0002DE9F74F0D4622F07F4402684FF4803760
:10C8F00005F150068F408046B60002EB8500C2F875
:10C900004873B6B2C2F80873D2F8041599464FF0CE
:10C91000000BD0F84035C0F8401542F806B05B1A5D
:10C920009259009223F07F43012B009A4FEA850A27
:10C930000CD1264B4FF4806043F001039847D8F8A0
:10C94000003043F806B09B590193019BD8F80010C2
:10C95000D1F80465C1F84473A31B23F07F43012B76
:10C960001CD11A4B05F5A875013443F0010341F8B9
:10C9700025404FF480609847D8F80030D3F804354C
:10C980009E4209D1D8F800300020C3F84473C3F8A0
:10C99000047303B0BDE8F08F0D20FAE78A44C9F1B3
:10C9A000FF13CAF84045D1F80405221A013A22F0D3
:10C9B0007F4203F57F439342EED3002AE2D1013454
:10C9C000CAF84045D1F804359842DAE7105402001D
:10C9D00003680222C3F8442309B1C3F80423704753
:10C9E00000684FF48271FFF707BF4FF4803303FAFA
:10C9F00001F10368C3F84813C3F8081370475031B6
:10CA00008900006889B2FFF7F7BE0368D3F8040510
:10CA10007047000090F9043001215A0903F01F0308
:10CA200001FA03F34032024941F82230704700BF57
:10CA300000E100E0024B034A1B681068184700BF82
:10CA4000D8270020D027002070B5064D06460024C8
:10CA500055F8043B0BB1304698470134042CF7D10C
:10CA600070BD00BFE8270020033082B240F2FE33E1
:10CA70009A42F0B51ED8114D00232E4628789FB259
:10CA800080B92C89B5F80AC064441444A4B2B4F542
:10CA9000806F07D80F80142101FB036359890A4472
:10CAA0005A81F0BD0133052B05F11405E6D148F29A
:10CAB0000660F6E748F20860F3E700BF1C28002094
:10CAC0000B4A0C4B5188142000FB0131CB6833B961
:10CAD0000420496810700122074801F09CB80749FA
:10CAE0000523137002238B80012209680023F3E7DA
:10CAF000002800201C2800200C26002020290020CF
:10CB000007B5002305490093054A0968054808232D
:10CB100001F053F803B05DF804FB00BF20290020AA
:10CB2000245402000C26002007B500230146009380
:10CB3000034A0448082301F040F803B05DF804FB01
:10CB40001C5402000C26002013B500230C46009351
:10CB50000146084A0848042301F02FF838B907496C
:10CB6000142303FB04140123237402B010BD48F204
:10CB70000D60FAE7185402000C2600201C28002043
:10CB800037B50A480A4B42689C88196853880325C0
:10CB9000033305709BB2002000909B0001EB8401E1
:10CBA000044801F00AF803B030BD00BF002800209F
:10CBB000202900200C26002010B50146044800F072
:10CBC000CCFE1C220446002108F070FB204610BD5C
:10CBD0000C2900204388033300EB830399420BD3D5
:10CBE00082884FF6FF739A4208D0038833B1806879
:10CBF000431C58425841704702207047012070473B
:10CC00002DE9F0410D460223154F2B80164600F505
:10CC1000805100F108044FF001088C420ED22368C5
:10CC200001330BD02046FFF7D5FF48B10EB186F88F
:10CC30000080022809D14FF480632B80BDE8F08189
:10CC4000A3683A68934200D93B602B88628803331B
:10CC500013442B806388033304EB8304DDE700BFB8
:10CC60001428002038B5144B14220D4602FB003066
:10CC70002B68446804F58051A3B15C88033403EB4E
:10CC800084048C4215D22368013312D02046FFF76A
:10CC9000A1FF012808D002280BD00028F1D12C6078
:10CCA000012038BD0834ECE76388033304EB8304C8
:10CCB000E7E70020F5E700BF1C280020426873B5B5
:10CCC00004460D4652B3224BD9688A4226D31B69CB
:10CCD0009A4223D812F0030320D11E490089098902
:10CCE00088421BD120689168884217D11A4C194696
:10CCF000606882428EB209D900F58050824205D226
:10CD00002E80B3FA83F0400902B070BD01310529CD
:10CD100004F11404ECD148F20963F2E700232B80FC
:10CD20001E460196288801A9FFF79CFF30B92B8881
:10CD300001339BB2042B2B80F3D9E5E7019B2268DA
:10CD400099689142EED16360024B1B892381DBE736
:10CD50000C260020002800201C2800202DE9F84384
:10CD60001C461D4B1B7806460F46154673B382B30F
:10CD70007CB3DFF86C804FF01409A388042B02D930
:10CD800048F2096020E009FB03F318F803302BB9DF
:10CD9000A0882146FFF766FF20B92060A3880133F1
:10CDA000A380EAE723681EB1998832889142EFD1C7
:10CDB0001FB119883A889142EAD19A68C5E90023DF
:10CDC000064B1B892B810020BDE8F88348F20160E7
:10CDD000FAE748F20460F7E7F8270020002800206F
:10CDE0001C28002008B5074B5888191DFFF73AFF8B
:10CDF00018B1BDE80840FFF7C3BEBDE80840FFF723
:10CE00005FBE00BF002800202DE9F04FA24FDFF8E1
:10CE1000AC9289B00646B8463B6823B99F4849465C
:10CE200000F0D5FD3860D8F8005029784B1E052B4E
:10CE300007D8DFE813F02200770077000901090125
:10CE4000600148F20E641422002103A808F02EFAB3
:10CE500041F61D539C4208BF0024D8F800300494CA
:10CE60001A78013A052A00F2F181DFE812F0DD01BB
:10CE7000E101010211021D0227022EB1884B00229E
:10CE80005A604FF40644DEE72B79032B18D8DFE80D
:10CE900003F010022631834B142101FB06F2D05C13
:10CEA000022813D19918002098544868FFF73CFED7
:10CEB00003E001232B71FFF723FE002800F0BE8062
:10CEC000774B00225A6048F20D64BCE70136052E0C
:10CED000E3D1734B01221A7000225A6002E17249B9
:10CEE0007248002302222B718A800968012200F017
:10CEF00092FEE2E76C4C00262E712068694DFFF728
:10CF000013FE6B4BD4F800C05A8814235343EA181D
:10CF1000EE5451682160A188C2F804C01181022238
:10CF2000A280CAE7B5F814A0AA7DDFF878B1AEB147
:10CF3000022AEB8806D9142101FB0AB1DA1C088900
:10CF400002440A81142202FB0ABAC3F57F43BAF8ED
:10CF50000A20FD331344AAF80A3092E7142303FB96
:10CF60000AB318895C6804EB8004062A69D8DFE8F4
:10CF700002F0274E36441D5A040041F61D54AA7D86
:10CF8000EB88022A06D9142101FB0AB1DA1C0889B0
:10CF900002440A81142202FB0ABAC3F57F43BAF89D
:10CFA0000A20FD331344AAF80A304CE741484249AD
:10CFB00000234360AB690360FFF780FE00285AD06E
:10CFC0000223AB75002300930423EA182146374857
:10CFD00000F0F3FD002831D048F20D64CFE72B6953
:10CFE000002B14BF03230123AB750023009305F12D
:10CFF0000C02042304F10801E9E70123AB750022C8
:10D00000EB8800922A699B0004F10C01DFE70329F9
:10D010000CBF05230623AB7500230093042305F101
:10D020000802E118D3E70623AB75234B1988214B7F
:10D030005868FFF789FD04460028A0D109B0BDE873
:10D04000F08F48F20E649AE7002E7FF41AAF2B7926
:10D05000012B35D0022B45D0002B7FF4F2AE0223FA
:10D060002B710DF10A01EB68039303A8CDE9046667
:10D07000FFF724FE10B948F20964E4E60498BDF80D
:10D080000A108388EB8003882B81FFF75DFD04463F
:10D09000002C7FF4D8AED1E7182800200C290020FE
:10D0A000F82700201C280020202900200C26002022
:10D0B00000280020DC2700202C2900201028002038
:10D0C0007F4B03AA3146A81DFFF748FE7C4B044660
:10D0D00058B999880498FFF737FD044648F2096368
:10D0E0009C42D5D141F61D54ADE608223146184682
:10D0F00008F0DCF8F2E7002E7FF4C3AE714BDA7B68
:10D10000B2B1DE731A78013A062A3FF69AAE01A14F
:10D1100051F822F0C1D10100EDD1010001D201008E
:10D1200007D2010043CE01000DD201001FD2010041
:10D130001A78072AE6D801A151F822F05DD1010042
:10D1400005D1010005D1010089D101009DD1010067
:10D15000BDD10100BDD1010085D101001A895A4815
:10D160005A4C01321A8100225A80DA73142505FBC9
:10D1700002F10132095DB1FA81F14909052A00F88D
:10D18000011BF4D1012207E051485968828849887F
:10D1900003320A44828002221A70B3E74B485A884D
:10D1A0004B49142505FB02020C685068086088880A
:10D1B0005460108102228A800622EDE70722EBE705
:10D1C000414A424C0020142512F8011B1FFA86FC2C
:10D1D00079B105FB064102F8010CD1F80CE0BEF173
:10D1E000000F06D1097C21B1A3F802C0FFF7FAFDB8
:10D1F0004DE70136052EE7D100221A705A806CE601
:10D20000FFF7BEFC43E7FFF75BFC40E72F4A5B8874
:10D21000142101FB03235868FFF786FC37E700223F
:10D220005A60FFF76DFC32E700238DF80C300DE0FB
:10D2300001228DF80C201A89ADF818209A88DB6835
:10D240000593ADF81A2000238DF81C3003A8FFF7D2
:10D25000FBFB002649461F48C8F8006000F0E2FBCF
:10D260001D48012100F08CFC00287FF4D5ADE5E6D7
:10D2700002228DF80C201A89ADF818209A88ADF892
:10D280001A20DA689B7D05929A1F53425341DBE7CF
:10D2900003228DF80C20DA88ADF818201A89DB6893
:10D2A000ADF81A200593D1E704228DF80C20DB8815
:10D2B000ADF818300023ADF81A30F3E70523B4E7D2
:10D2C00030290020002800200A2800201C280020E7
:10D2D000202900200C2900201C2900204068FFF78D
:10D2E00093BD000008B50548012100F031FC18B9D4
:10D2F000BDE80840FFF788BD08BD00BF1C2900201D
:10D300002DE9F3419846374B1B7806460D46002B16
:10D310005CD000295DD009884FF6FF7399425BD03D
:10D320006B88002B58D06B689B0758D14AB92F895E
:10D330000DF102013846FFF797FB30B102B0BDE8AE
:10D34000F08113885788ADF8023001A8FFF734FC4C
:10D35000044660B9BDF80230234A142101FB0323BF
:10D3600058890338C01B588148F20760E6E780F807
:10D37000008000238375BDF8023083826B680361EF
:10D3800001211A4800F0F0FB2B882381B8F1030F2C
:10D390006B88A38004BF0423A3754FF0000508BF6A
:10D3A0003368E06008BFA3611148E780658101A987
:10D3B00000F0FDFA36B1E36833600E4B75601B89EF
:10D3C000B5723381FFF78EFF0020B7E748F20160A6
:10D3D000B4E748F20460B1E748F20360AEE748F210
:10D3E0000260ABE7F82700201C280020142800204A
:10D3F0000C2900200028002008B5034607480268D1
:10D40000042A08D00168064A42F82130012100F0C0
:10D41000ABFB002008BD48F20B60FBE72829002089
:10D42000E82700202DE9F04F89B01422002103A83D
:10D4300007F03CFF774A1378914603F0FF0B3BB1AE
:10D4400003A8FFF701FB0026304609B0BDE8F08FC6
:10D45000101D00F0A1FB0028F5D140F6F8734FF045
:10D4600080521B685C1C08BF6B4B6C4C08BF1B6870
:10D4700011695269581C08BF02FB01F32361684916
:10D48000A3F5C04300222046E36000F088FB01942E
:10D4900006460028D8D163496348644F1C238C2278
:10D4A00000F026FAB04635464FF0060A3446019B96
:10D4B000D86858F8003018EB00002DD05C4A934231
:10D4C00040F0A68043685B4A934213D001329342F6
:10D4D00027D1594BBBF1000F5FD15849186000228A
:10D4E000FFF78EFB544B9B88022B0CBF04230823B1
:10D4F0001D4335E0142161437B1800227A5401F169
:10D500001002083158603A443944FFF779FB45F07E
:10D5100002050134A4B223E05A1C02D0444A9342CB
:10D5200030D1031D00F580511A6801322AD104332D
:10D530009942F9D1404B1A682AB9022218609A80A0
:10D540004FF0010B0AE0142363430221FA18F95447
:10D550003B4B50605C8001341181A4B245F0010561
:10D5600008F58058B8F5C04FA1D1BAF1010F98BFA6
:10D570000025EDB2022D02D0062D1ED03DBB48F293
:10D580000A6661E714236343FA180AF1FF3A506010
:10D590000322FA541FFA8AFABBE714226243B9182D
:10D5A0004FF0020C07F802C01A684A60244AA1F83A
:10D5B00008C054800134A4B28FE7012389F80030F9
:10D5C00003A80023C9F80430FFF73EFA3CE702A89D
:10D5D000FFF7F2FAC8B10123013D03700A2D09D803
:10D5E000DFE805F006080608070807080F110F0016
:10D5F0000023037102A90C4800F0D9F9FFF772FE6D
:10D6000022E70323F5E70223F3E748F207661BE767
:10D61000013385E7F8270020141000100C260020A5
:10D6200038540200802800200C2900201C280020EB
:10D63000DEC0ADDEFE011EF12029002024290020DD
:10D640000028002073B50D460446C8B1C1B10DF1E4
:10D650000601FFF733FBB0B10C4BBDF8060066685E
:10D66000142202FB003001210C3000F07DFA6368C7
:10D670002E600C336B600123A372002002B070BDDA
:10D6800048F20460FAE748F20960F7E71C28002036
:10D6900013B50446A8B10DF10601FFF70FFB98B1D1
:10D6A0000C4ABDF80630142101FB0323DA6872B17D
:10D6B000A27A62B1DA680020013ADA60A07202B0A0
:10D6C00010BD48F20460FAE748F20960F7E748F253
:10D6D0000560F4E71C28002002230022FFF710BE9B
:10D6E00018B103230022FFF70BBE48F20460704715
:10D6F000114B1B7813B50446ABB14FF6FF7398423C
:10D7000014D001A8FFF758FA98B10523037001233C
:10D710000371C48001A9094800F049F9FFF7E2FD4F
:10D72000002002B010BD48F20160FAE748F2036041
:10D73000F7E748F20760F4E7F82700200C290020FB
:10D740000F4B1B7807B5A3B101A8FFF735FA98B1C5
:10D750000623037001A90B4800F029F90A4B1A7837
:10D760000AB10122DA73FFF7BDFD002003B05DF8B6
:10D7700004FB48F20160F9E748F20760F6E700BFF2
:10D78000F82700200C2900200028002007B5ADF85C
:10D790000600ADF804100DF1060001A9FFF7DEFA4E
:10D7A00003B05DF804FB07B51346ADF806000A4662
:10D7B00000200DF10601FFF7D1FA03B05DF804FB7C
:10D7C00007B51346ADF806000A460DF10600002124
:10D7D000FFF7C4FA03B05DF804FB20B119B1036888
:10D7E0000B600020704748F2046070472DE9F84F45
:10D7F0003B4B1B780446002B6BD000286CD01222C8
:10D80000002107F053FD374EDFF8E0B006232380F8
:10D81000354B0027B1464FF014084FF0010A7589C7
:10D82000328971682A4492B231B10868984203D1B2
:10D8300048685844012802D920880138208008FB14
:10D840000790B4F802C0C068604460802089054435
:10D850006089258110446081C2F58062A08992B2FE
:10D86000904201F1080538BFA28101F58051A9421B
:10D8700027D92A68013224D02846FFF7ABF90128BE
:10D88000194B07D0022812D00028F0D1A28801320B
:10D89000A28007E0E2880132E280E28968880332F0
:10D8A0000244E2816A88033205EB8205DFE7E28801
:10D8B00084F810A00132E280E289491B02EBA10149
:10D8C000E1810137052F06F11406A8D10020BDE83B
:10D8D000F88F48F20160FAE748F20460F7E700BF0A
:10D8E000F82700201C280020DEC0ADDE02FEE10E7D
:10D8F00010B561B1B2FBF3F403FB1424A4B244B934
:10D90000C0E9001484608281C381204610BD0E20CE
:10D91000FCE70920FAE782B050E8022FC188B2EB99
:10D92000324F4FF0000317BF92B241EA014142EA81
:10D93000014104E04268B2EB324F08BF012340E8E6
:10D940000212002AE8D18DF807309DF80730002B2D
:10D950000CBF1120002002B0704737B550E8013FDE
:10D960009DB2C48925448489A54228BF2D1B048902
:10D97000A54202BFBFF32F8F002207E0C5EA0305CF
:10D9800040E80154002CE9D14FF001028DF803204A
:10D990000193019B9DF803200B6002F0FF0322B16D
:10D9A0000B880068184403B030BD1846FBE70A88AE
:10D9B0004B889A4209D150E8012FC2EA024240E85E
:10D9C0000123002BF7D1012070470020704737B5A5
:10D9D00050E8023F1FFAA3F5C488A54202BFBFF377
:10D9E0002F8F00220DE0C48925448489A54228BFD9
:10D9F0002D1BC3EA054540E80254002CE8D14FF046
:10DA000001028DF803200193019B9DF803200B6018
:10DA100002F0FF0322B14B880068184403B030BD08
:10DA20001846FBE70A884B889A4209D150E8022F32
:10DA3000C2EA224240E80223002BF7D101207047BE
:10DA40000020704701F01F024B090121914000EBBB
:10DA5000830000F065B84B0910B501F01F040121E7
:10DA6000A14000EB830000F04FF8E04000F001001F
:10DA700010BD01F01F0301229A404B0900EB830007
:10DA8000D14300F059B84B0901F01F0150F82300B1
:10DA9000C84000F0010070472DE9F0474F1E7F0994
:10DAA00080460E460137002558F8254008EB8509C9
:10DAB000E44394FAA4F4B4FA84F44FEA451A202C0F
:10DAC00006D10135AF42EFD834462046BDE8F08795
:10DAD0005444A642F5D921464046FFF7BCFF002832
:10DAE000F3D0D9F80040E44394FAA4F4B4FA84F4EF
:10DAF000E5E710B5034653E8000F0A4643E8002463
:10DB000094F0000FF7D110BD10B5034653E8000F95
:10DB100040EA010243E8002494F0000FF6D110BD62
:10DB200010B5034653E8002F42EA010043E8000421
:10DB300094F0000FF6D110BD10B5034653E8002F46
:10DB400002EA010043E8000494F0000FF6D110BD92
:10DB500010B5034653E8000F00EB010243E8002430
:10DB600094F0000FF6D110BD10B5034653E8002F16
:10DB700002EB010043E8000494F0000FF6D110BD61
:10DB800010B5034653E8002FA2EB010043E8000460
:10DB900094F0000FF6D110BD0121FFF7B5BF0B4681
:10DBA00010B4114628B123B103605DF8044B1B6823
:10DBB00018470E205DF8044B70472DE9F04108B37B
:10DBC00002B3D0F800E0BEF1000F1ED0FBB14568F3
:10DBD000D5F80480B3FBF8F508FB1535BDB942EA6A
:10DBE000010C1CF0030F14D1C568A94211D34D1EBE
:10DBF000EC180569AC420CD8DEF80C40A446BDE830
:10DC0000F04160470E20BDE8F0810820FBE70920C5
:10DC1000F9E71020F7E7F0B5D8B1D0F800C0BCF1B3
:10DC2000000F18D0CAB14768D7F800E00EF1FF37EF
:10DC30000F4214D1C768B94211D304694D1E0EFBBF
:10DC40000255A5420BD8DCF81040A446BDE8F040D0
:10DC500060470E20F0BD0820FCE70920FAE71020FD
:10DC6000F8E729DF704728DF704770B503689E68C2
:10DC700086B004460D466EB114220021684607F0B6
:10DC800015FBA3680593237901952BB1012B0DD0CA
:10DC90006846B04706B070BD01238DF80030236997
:10DCA0000293E368039363690493F1E702238DF819
:10DCB0000030E3681B030293F5E708467047002035
:10DCC00070470000024B187A003818BF01207047D7
:10DCD000D4290020034B187A0122B0FA80F05A743C
:10DCE00040097047D429002008B510461A4607F0AD
:10DCF000B4FA002008BD000008B514220021044831
:10DD000007F0D4FA0348FFF706FE002008BD00BF65
:10DD1000D4290020C429002010B5094C094B4360C8
:10DD20002046FFF739FF40B906F034FC064920745D
:10DD30001C2306488C22FFF7DBFD002010BD00BF2E
:10DD4000D42900202C54020038290020C4290020A6
:10DD500070B5244C244E237A25463BB923492448E8
:10DD6000FFF735FE306008B9606070BD022334688B
:10DD70002B72237973B1012B24D020460321FFF7A6
:10DD800074FF00232B726B6018491948BDE870407E
:10DD9000FFF748BED4E90523D21AB2F5805FD4E973
:10DDA000031028BF4FF480529208012A38BF012285
:10DDB00019441844FFF755FF50B11128DDD1012354
:10DDC0002B72D2E7D4E903031844FFF74CFFF3E7C3
:10DDD0002B7C002BC9D10146BDE87040022000F029
:10DDE00009B800BFD4290020EC290020E829002030
:10DDF000C429002038B5831E012B45D8234C237A33
:10DE0000002B41D0022B09D1032830D0204B002217
:10DE10001B68E2601A793AB1012A22D0637C7BBB8D
:10DE2000BDE83840FFF794BFD3E905128D1AB5F568
:10DE3000805F94BF521902F580529A619142EDD1F0
:10DE400002284FF0000308BF19462372104B18BF79
:10DE50000D211868FFF709FF0E490F48FFF7E2FD93
:10DE6000DCE71A6901321A615B699A42E7E7E36805
:10DE70000133082B01D8E360D0E70023E360DFE73C
:10DE8000BDE8384006F076BB38BD00BFD42900207D
:10DE9000EC290020E8290020C429002000F0FD031F
:10DEA000012B08D1044B00225A74421E50425041AB
:10DEB0001874FFF74DBF7047D429002010B5064CE9
:10DEC000201DFFF769FE28B9637C1BB9BDE810402F
:10DED000FFF73EBF10BD00BFD42900202DE9F3415C
:10DEE00080460D460F4801A916461F46FFF735FD2F
:10DEF0000446A8B11C22002107F0D8F92D0B0123FC
:10DF0000237101A90748C4F80080A760E560666135
:10DF1000FFF74DFDFFF7D2FF002002B0BDE8F08112
:10DF20000420FAE7C42900202DE9F74381468846FA
:10DF3000104801A917461E46FFF70FFD0446B0B171
:10DF40001C22002107F0B2F900250A9BA36001A959
:10DF5000C4E9037807482571C4F800906661FFF7AB
:10DF600026FDFFF7ABFF284603B0BDE8F083042091
:10DF7000FAE700BFC429002033DF704741DF704754
:10DF80000D4A08B5002313700C4A1360BFF35F8F6E
:10DF90000B490C4800F0A0F80B4A0C480121FEF791
:10DFA000F1FA024630B9BDE8084009484FF4804113
:10DFB000FEF7F3BA08BD00BF202A0020242A002063
:10DFC0005C540200F0290020C5E001005854020012
:10DFD000002A002007B500230DF107008DF8073057
:10DFE000FEF7D0FBF1EE103A23F09F03E1EE103A7A
:10DFF000BFF35F8F094B4022C3F884219DF80700CF
:10E00000FEF7E4FB06F0C6FA20B1FFF7B7FF03B056
:10E010005DF804FB20BF40BF20BFF8E700E100E04F
:10E0200070B5224D044601212846FFF762FDBFF37B
:10E030005F8F2E4638B9042C0AD01D4B1A781AB1BE
:10E04000BFF35F8F286070BD1A4A147001221A70E6
:10E05000194C184D636828787BB90238012813D809
:10E06000BFF34F8F1549164BCA6802F4E0621343A1
:10E07000CB60BFF34F8F00BFFDE71B68984788B1A7
:10E08000204600F033F8E5E706F084FA08B1FFF720
:10E0900073FF4FF080430122C3F80025BFF34F8F79
:10E0A00020BFFDE7BFF35F8F3060CCE7242A00205C
:10E0B000202A0020F8290020F029002000ED00E0AF
:10E0C0000400FA05034B1B7813B10420FFF7A8BF27
:10E0D000704700BF202A00200B684A6843609342C3
:10E0E00008BF0023016008BF43607047436843B125
:10E0F0000268916852680B449342436004BF002356
:10E100004360704770B5446806460D46206818B1F4
:10E11000B3682946984718B923682B60256070BDFD
:10E120002468F3E74368186808B102681A6070470A
:10E130004368186870474368186800B97047884298
:10E1400003D102681A600120704703460068F4E7B3
:10E150000178036AC26821B1C3F80C25002343701B
:10E160007047C3F80825F9E738B5037D0446002B4E
:10E170003FD18369DBB9E378A2789A421FD1207836
:10E18000236AE168C0B1C3F8081501230532637042
:10E1900022612379022B0ED1E36921691868224696
:10E1A000FEF7FBF938B1BDE83840FEF715B99847DE
:10E1B0002379022BDFD038BDC3F80C15E5E733B95E
:10E1C0002046FFF7C5FFA37805332361E1E72578F3
:10E1D000216AE06855B1C1F8080513FB02F31B1270
:10E1E00001210533617023612175D2E7C1F80C0567
:10E1F000F3E7FFF7ADFF0023C278037583789A1A1F
:10E2000053431B12E0E7000070B58D680B78037074
:10E21000C0E902554B68826103624B788370044603
:10E22000C868104AE0610021FEF7ACF940B90E4E13
:10E23000032135B92046FFF78BFF012323712846C0
:10E2400070BDEB070BD51F288BBF00F01F030346E3
:10E2500032464FF0A04203F5E07342F8231001303C
:10E260006D08E6E769E1010000030050022370B584
:10E270000371C16004460D46FFF76AFF8168866935
:10E2800029430025816005758561FFF76DFFA66153
:10E29000284670BD38B5C36904461868FEF795F97D
:10E2A00005462046FFF754FF0DB901232371284688
:10E2B00038BD83788B4226BFC1700020072070478D
:10E2C000BFF34F8F0549064BCA6802F4E06213435F
:10E2D000CB60BFF34F8F00BFFDE700BF00ED00E054
:10E2E0000400FA050A4B1B685A1C05BF094B0A4A71
:10E2F0000A4A10680ABF1B781068C0F303100D2B80
:10E3000004D101288CBF00200120704700207047F5
:10E3100030010010E00F00F0E80F00F034010010B1
:10E3200008B5FFF7DFFF40B14FF080430022C3F88C
:10E330000C21C3F81021C3F83825FFF7D3FF0028BC
:10E3400046D04FF08052594BD2F80414C3F8201530
:10E35000D2F80814C3F82415D2F80C14C3F8281501
:10E36000D2F81014C3F82C15D2F81414C3F83015D1
:10E37000D2F81814C3F83415D2F81C14C3F8401599
:10E38000D2F82014C3F84415D2F82414C3F8481561
:10E39000D2F82814C3F84C15D2F82C14C3F8501531
:10E3A000D2F83014C3F85415D2F83414C3F86015F9
:10E3B000D2F83814C3F86415D2F83C14C3F86815C1
:10E3C000D2F84014C3F86C15D2F84424C3F8702571
:10E3D000FFF788FF48B14FF08043D3F80024D107FE
:10E3E00044BF6FF00102C3F80024314AD2F88830EC
:10E3F00043F47003C2F88830BFF34F8FBFF36F8FC1
:10E400004FF01023D3F80C22D2071ED5294B01223E
:10E41000C3F80425D3F80024002AFBD04FF01022C3
:10E42000D2F80C3223F00103C2F80C32214B1A4609
:10E43000D3F800140029FBD00021C3F80415D2F84A
:10E440000034002BFBD0FFF73BFFD3F80022002A5B
:10E4500003DBD3F80432002B23DA164B0122C3F876
:10E460000425D3F80024002AFBD04FF010221221FB
:10E47000C2F80012D3F80024002AFBD04FF010237A
:10E480001222C3F804220B4B1A46D3F800140029B9
:10E49000FBD00021C3F80415D2F80034002BFBD0C8
:10E4A000D1E7054B054A1A6008BD00BF00C0004017
:10E4B00000ED00E000E00140282600200090D0039D
:10E4C00038B5074C051E04F1080318BF1C46236825
:10E4D0002BB11A6822605B6828469847F7E738BD79
:10E4E000302A002020B9054B01225A70FFF7E8BFFF
:10E4F000012802D1014A9070F8E77047282A0020CD
:10E5000020B9034B01225A70FFF7DABF704700BFF2
:10E51000282A002038B50B4C237883B90A48636059
:10E52000A3602361E36000F097F8054606F032F837
:10E5300008B900F09DF801232370284638BD8525D1
:10E54000FBE700BF282A0020E5E4010037B5184C9E
:10E55000A378054603F0FF029BB110B14368012088
:10E56000984700230DF107008DF80730FEF70AF9F0
:10E57000E3689DF807000133E360FEF727F903B075
:10E5800030BD0DF107008DF80720FEF7FBF825B12F
:10E59000226913463BB92A602561E368002BE7D165
:10E5A00000F07CF8E4E79D42F7D01B68F2E700BF7B
:10E5B000282A002037B50B4C00230DF107008DF8F9
:10E5C0000730FEF7DFF8E368013BE360E56815B963
:10E5D00000F076F8A5709DF80700FEF7F7F803B095
:10E5E00030BD00BF282A0020012813B508D0032819
:10E5F0001CD018B9104B0122C3F8802002B010BD06
:10E600000E4C00230DF107008DF80730FEF7BAF825
:10E6100023780BB9FFF77EFFE3689DF8070001330D
:10E62000E3600123A370FEF7D1F8E7E700F020F8DC
:10E63000FFF7C0FFE2E700BF00E100E0282A00206A
:10E6400008B505F0A7FF28B94FF08043D3F81804A8
:10E65000C0F3004008BD0000044A137923B901212A
:10E660001060117118467047852070473C2A0020C1
:10E67000084B1A68D2075FBFC02283F8002301222B
:10E680001A604FF080420123C2F81835024A137015
:10E69000704700BF00E100E0442A0020074B002241
:10E6A0001A6082B01B680193019B4FF080430222E5
:10E6B000C3F8042301229A6002B0704704010040AD
:10E6C000044B01221A604FF08042D2F81834DB0369
:10E6D000FBD470470C00004000F1804000F5C040C2
:10E6E000002382B0036003680193019B02B070476E
:10E6F00003681F2B83BF03F01F03036001484FF023
:10E70000A04070470003005007B5019001A8FFF733
:10E71000EFFF019B00EB8300D0F8003723F4403378
:10E72000C0F80037D0F8003743EA0141C0F80017BD
:10E7300003B05DF804FB0000054B4FF0FF320728E3
:10E7400043F8202084BFC01880F85220704700BFD3
:10E75000482A002010B5174C94F8643043BB04F1EC
:10E7600030032A21FF22013911F0FF0103F8012BA8
:10E77000F9D1C8B2FFF7E0FF01310C29F9D1062227
:10E7800000210D4806F092FD0C4BC02283F80623B1
:10E7900040221A604FF4BE70FFF79EFF084B4FF007
:10E7A0000042C3F80423012384F86430002010BD24
:10E7B0000820FCE7482A0020A62A002000E100E00B
:10E7C0000060004037B5354B1A18044692F9300006
:10E7D000013061D18878002852D01846002250F8C4
:10E7E000045B013546D1181980F83020002043F829
:10E7F0002200920002F1804202F5C0420B78D2F86A
:10E800001055487825F499151B04000525F4F85592
:10E8100000F4801003F44033C2F810550343200283
:10E82000D2F8105500F47C5003432B43C2F8103546
:10E830004A780194012A01A826D1FFF759FF019BCC
:10E840009A40C0F8082501A80194FFF751FF019BE9
:10E85000134903F5E073032240F8232024FA02F25F
:10E86000012304F0070003FA00F08B5C184388547E
:10E87000002003E00132082AB1D1042003B030BDEA
:10E88000FE2382F83030D3E7FFF732FF019A0123ED
:10E890009340C0F80C35D6E70820EFE7482A00205F
:10E8A000A62A0020F7B53B4E3318054693F93030C1
:10E8B000002B6CDA8B78C3F34003002B0BBF0824CA
:10E8C00000240C200820844202D1042003B0F0BDB3
:10E8D00056F82470013743D1701946F8242080F887
:10E8E000304013B9331983F852508B785A0717D434
:10E8F000D80737D501A80195FFF7FAFE019B00EB79
:10E900008300D0F8003723F00203C0F80037224814
:10E91000EA0805F007070123BB40875C3B438354AB
:10E920008B780A7813F0020328D0A40004F1804405
:10E9300004F5C0442D02D4F8103523F44F3323F4EA
:10E940004073C4F810351204D4F8103505F47C5522
:10E9500002F4403215431D43C4F810550020B5E7BA
:10E960000134B0E701A84A780195FFF7C1FE019B89
:10E9700003F5E073920040F82320C8E7083C3444D4
:10E9800094F85A5045EA821284F85A20E6E70820A3
:10E990009CE700BF482A0020A62A002073B5224C1D
:10E9A0002618054696F93020072A1ADD224492F8E7
:10E9B00052309B09032B0FD1019001A8FFF798FE5D
:10E9C000019BD0F81015D94001F001010231284611
:10E9D000FFF79AFE02B070BD012B0CBF022103218C
:10E9E000F5E7D3B2072BF5D8930003F1804303F585
:10E9F000C043D3F8100540F00100C3F8100502F140
:10EA00004000800080B2FFF767FE0029E2D096F94F
:10EA1000303054F82330002BDCD0012303FA02F20B
:10EA2000024BC3F80423D5E7482A002000600040C9
:10EA30002DE9F04F002489B0CDE90244624D4FF436
:10EA40008072012102F1804303F5C04390B21B683C
:10EA5000012B06D1D5F804330B4202D0FFF73CFE60
:10EA60000C430432B2F5907F4FEA4101EAD1574B93
:10EA70001B68012B0ED14FF4BE70FFF72DFE4FF037
:10EA8000A04344F00044D3F810350293504BD3F820
:10EA90001035039314F0FF0F1AD04E4F01260025B6
:10EAA000264210D0AB0003F1804303F5C043D3F8F6
:10EAB0001005D3F8101557F8253023B1C1F30141E3
:10EAC000C0F3052098470135082D4FEA4606E7D1E7
:10EAD000002C75DA04AF002304937B604FF0FF3302
:10EAE000CDE90633DFF8EC90DFF8EC8000252E4608
:10EAF00018F9012B531C4AD0C2F3C2000123D4B22F
:10EB000002F03F0B02F0070203FA02F208AB1918F9
:10EB100011F8083C13423AD009EB0B03A40993F90E
:10EB2000303059F823A0BAF1000F08D1032C2ED1B0
:10EB300017F800C04CEA020C07F800C001E0032CF3
:10EB4000F6D001A8CDF804B0FFF7D2FD019B11F873
:10EB5000181C03F5E07C114250F82C00C0F3014072
:10EB600005D0022813D1032C0BD1214604E0032841
:10EB70000DD1032C05D102215846FFF7C5FD013503
:10EB8000EDB2BAF1000F02D021465846D047013607
:10EB9000042EADD1A5B14FF0A0430299D3F81025B2
:10EBA00003F540739142D3F8103502D1039999428D
:10EBB00006D002920393049A059B0692079393E76B
:10EBC00009B0BDE8F08F00BF006000407C610040EC
:10EBD00000030050482A0020A22A0020014B1B6895
:10EBE000184700BFB02A002013B5064C23683BB17C
:10EBF000054B1B6898470023236023680193019B02
:10EC000002B010BD00010140BC2A002070B5114BBC
:10EC10001960114B1C780546D4B9104E01221A70A8
:10EC20000378C6F80C3541684FF47A720023C803A4
:10EC3000490C06F06DFAC6F804052B7A084A5B0108
:10EC4000DBB282F810334FF480331360204670BD7E
:10EC50000820FCE7BC2A0020B92A0020000001405F
:10EC600000E100E0044B0122C3F804231A60034BC7
:10EC700002221A70704700BF00000140B92A00202C
:10EC800037B5054600240DF107008DF80740FDF764
:10EC900079FD0C4B1A78072A11D8511C19700A49B2
:10ECA0002A70D1F80805012393400343C1F80835C1
:10ECB0009DF80700FDF78AFD204603B030BD04240F
:10ECC000F6E700BFB82A002000000140034B044AC9
:10ECD00000F5C07043F82020704700BF00000140DD
:10ECE0003546526E00F1804000F5E040002382B0CE
:10ECF000036003680193019B02B07047F0B5504B6D
:10ED0000504C1B6885B0002B3DD04FF4827094F8B6
:10ED10002E20FFF7E7FF2AB394F82F3013BB4A4B9E
:10ED20001B68002B33D04FF48070FFF7DBFF638B41
:10ED300094F82D108B424FD922895B1A9BB292B264
:10ED40006383D31A626802EB4303404AC2F82C364D
:10ED5000C2F830164FF48270FFF7C4FF3C4B01221B
:10ED60001A6014E0636802932389ADF80C30E368FD
:10ED700000218DF8041023BB2374236801A8984751
:10ED8000002384F82F3094F82E30002BC7D1314B5C
:10ED90001B685BB14FF48870FFF7A4FF0023237456
:10EDA00002238DF8043001A8236898472A4B1B687A
:10EDB000EBB14FF48A70FFF795FF0023237405B081
:10EDC000F0BD208B608363602081E160002AD4D194
:10EDD0001E4B01221A60D0E7BCD1E368012284F8FF
:10EDE0002F2013B100226283AFE76383B2E7666925
:10EDF0004FF000470125002EE1D0B6FA86F227FA3F
:10EE000002F34632920026EA030602F1804303F53C
:10EE1000E0431B68002BEED01046FFF763FFA2F51E
:10EE20008C72D30882F00402C2F380028DF808309D
:10EE30008DF8045023688DF8092001A89847DAE777
:10EE400004710040C02A00200071004000700040A2
:10EE500004700040107100401471004038B51E4B22
:10EE6000044693F82C00A8BB1C4A19602178C2F80C
:10EE7000F0156178C2F8F415E5781874012183F86B
:10EE80002C1083F82D00586183F82F0083F82E5042
:10EE90006FF00043C2F808334FF48270FFF722FF8F
:10EEA0004FF48070FFF71EFF4FF48A70FFF71AFFD0
:10EEB000A3780B485B01DBB280F807338023036043
:10EEC0000223C2F804330DB1C2F80413C2F80015CE
:10EED000002038BD0820FCE7C02A00200070004058
:10EEE00000E100E030B5224B1A7C002A3ED100F14F
:10EEF0000C0403EB4402127922B993F82D2001325D
:10EF000083F82D2003EB4403CA790C7A8D781A71AB
:10EF10005C714B782D021B0105F4E06503F03003B2
:10EF20002B430D7805F003052B43CD782D0305F415
:10EF300080552B430D792D0405F4E0252B434D79A5
:10EF400089792D0505F48015090601F080712B43A0
:10EF50000B43010101F1804101F5E0410020C1F8BE
:10EF60001835C1F81445C1F8102530BD1120FCE753
:10EF7000C02A002070B5344A147C04F0FF03002C32
:10EF80005FD1324C012503261574C4F80863C4F818
:10EF90002C16C4F8305692F82D10A9420CD91C46F4
:10EFA000190101F1804101F5E0410133082BC1F85D
:10EFB0001445C1F81045F3D100F10C03000102EB38
:10EFC000430300F1804000F5E04019795B79C0F817
:10EFD0001435C0F810151D4901230B604B6042F237
:10EFE000107301F58271086808B9013BFBD14FF439
:10EFF0008070FFF777FE4FF48270FFF773FE92F890
:10F000002D30012B11D9104800210B0103F1804351
:10F0100003F5E0430131047F457FC3F81455082907
:10F02000C3F8104500F10200EFD192F82E10074B03
:10F0300029B103210020C3F80413107470BD02210C
:10F04000F8E71120FAE700BFC02A00200070004056
:10F05000F0B51B4F8BB207EB001443EA0243C4F830
:10F060001C35184B40005C6900F1010C4FF0004664
:10F0700011F5006F26FA0CF64FF0800505FA00F541
:10F080000BBFB44334435C615C610CBFC7F80853E9
:10F09000C7F8045340244FF000455969844025FACD
:10F0A00000F040F2FF75AA42054A0BBF81430143BD
:10F0B000596159610CBFC2F80843C2F80443F0BD5E
:10F0C00000700040C02A002010B5124B1A7CF2B923
:10F0D00000F10C0103EB4102127922B193F82D20CB
:10F0E000013A83F82D2003EB410300249C800301A7
:10F0F00003F1804303F5E0430749C3F8144540F2A8
:10F10000FF72C3F81045FFF7A3FF204610BD112082
:10F11000FCE700BFC02A002000F8FFFF38B5134B02
:10F120006FF00042C3F80823114A8021C2F8801012
:10F13000104A01211160104942F21072086808B9A2
:10F14000013AFBD10D4D0024C3F800452C7405EBAA
:10F1500044031B7F13B1E0B2FFF7B6FF0134082C64
:10F16000F5D1002385F82C3038BD00BF0070004079
:10F1700000E100E00870004014710040C02A002047
:10F180000023435082B043580193019B02B0704763
:10F19000F0B51C4B45791C4C43F8252005EB450385
:10F1A0006F00E35C63BB90F9046003798A78002EFA
:10F1B000ADBF06F1604CDFF854C003F00F0E0CF544
:10F1C000614C4FEA4212D2B2B4BF0CF80E208CF858
:10F1D000002376090122DFF838C003F01F0302FA8A
:10F1E00003F34CF8263003680888C3F808053D444B
:10F1F000631908796255C978587099700020F0BD7C
:10F200000820FCE7F42A0020F02A002014ED00E09A
:10F2100000E100E0036801221A604379024A03EB2F
:10F2200043030221D1547047F02A00202DE9F04118
:10F23000224E234FDFF88C8000244FF48035D7F81E
:10F240000433A6F580412B4289B20CD0336853B108
:10F25000C7F848533846C7F80853FFF791FFD8F866
:10F260000030E0B298470134042C4FEA450506F11E
:10F270000406E4D11248D0F80433DA070AD5D0F8EE
:10F2800000313BB14FF48071FFF77AFF0D4B204600
:10F290001B6898470A48D0F804339B070CD5D0F870
:10F2A00004314BB14FF48271FFF76AFF054BBDE8A3
:10F2B000F0411B6805201847BDE8F081404102403D
:10F2C00000400240F42A0020BFF34F8F0549064B4F
:10F2D000CA6802F4E0621343CB60BFF34F8F00BFF4
:10F2E000FDE700BF00ED00E00400FA0574DF7047A1
:10F2F00076DF704778DF70477ADF70477CDF7047D2
:10F300008FDF704767DF704734DF704735DF704746
:10F3100033DF70473FDF704770477047704700002A
:10F3200002784368052A08D8DFE802F003080807D6
:10F33000070C13B9054B01221A707047002BFCD142
:10F34000034BF8E7002BF8D1024BF4E7A52F002080
:10F3500010300020BC2F00207047052001F0E4BBD6
:10F3600008B5074B0748002240F266611A60FDF7B6
:10F3700014F918B1BDE80840FDF72EB808BD00BF6C
:10F380001C300020302B0020FDF726B80388212BED
:10F3900013B5044646D007D8112B0ED0152B49D0F3
:10F3A000102B1CD002B010BD3B2B01D0562BF9D135
:10F3B000A0881321FFF79CFF2FE0224C224B2088CE
:10F3C00000221A704FF6FF729042EBD003F066FFF6
:10F3D00008B1FDF701F84FF6FF732380E2E71B4BFE
:10F3E0001B788BB11A48FDF7F0F808B1FCF7F4FF71
:10F3F000032001F099FB174800224FF42031FDF75C
:10F40000CCF808B1FCF7E8FF0F4BA18812480122A5
:10F410001A70124B198003F09BF90028C2D0FCF738
:10F42000DBFFBFE7002369468088ADF80030FFF7B7
:10F4300067FFF2E700F108010622684605F00DFFBC
:10F44000B0E700BF32260020202B00206C300020C7
:10F45000002B0020A0300020C02F002030260020EC
:10F4600010B5034C237803B110BDFEF7B3FDF9E7E7
:10F4700010300020104B10B51988104C89B220466E
:10F4800001F0E5F90E4B1988204689B201F016FA11
:10F490000C4B2046196801F048FA0B4B20461968BE
:10F4A00001F078FA094B1988204689B201F0A7FAD1
:10F4B000074B00221A7010BD282B0020CC2F0020F3
:10F4C000FC2A0020C8300020242B00202A2B0020FA
:10F4D0001130002010B5064C23783BB1012001F01B
:10F4E00023FB237883F00103237010BD0520F6E78A
:10F4F000C5300020084B1B7810B54BB1074C237862
:10F500003BB1032001F010FB237883F0010323704B
:10F5100010BD0520F6E700BF6C300020C43000208D
:10F52000032808B50AD1064800224FF40051FDF720
:10F5300034F818B1BDE80840FCF74EBF08BD00BF65
:10F54000002B002008B503784BB9054B3B211888E8
:10F55000FFF7CEFE18B1BDE80840FCF73DBF08BD7F
:10F560003026002030B5324A324D137885B0002B5A
:10F5700059D101231370304A8DF80030106851685A
:10F58000127A4FF48373ADF8023001AB03C32B49F9
:10F590001A706846FFF762FC08B1FCF71DFF01A96D
:10F5A0000020FFF79FFC08B1FCF716FF2448FDF789
:10F5B0000CF808B1FCF710FF2248FDF706F808B177
:10F5C000FCF70AFF022001F0AFFA1F4B1F48196831
:10F5D000013119601E4B00242C601C601D4B1C80E7
:10F5E0001D4B1C801D4B1C801D4B1C601D4B1C604B
:10F5F0001D4B1C601D4B1C601D4B1C7001F0F2F874
:10F60000FCF7EEFF1B4B1C49186022461B48FCF719
:10F61000C4FF04461A48FCF7D8FF14B12046FCF793
:10F62000DBFE05B030BD2B6801332B60F9E700BF6E
:10F63000743000201C300020885402001DF30100AB
:10F6400078300020002B002060300020CC2F0020DC
:10F650002C2B00202A2B0020282B0020FC2A002005
:10F66000C0300020242B0020F82A0020C8300020C1
:10F670006C30002070300020CD2C0100502B002079
:10F68000A030002008B50548032101F0BCFD18B1E9
:10F69000BDE80840FCF7A0BE08BD00BF702B0020ED
:10F6A00013B5044603F0B9FF204604F096F820464F
:10F6B00003F0C0FF23780C2B0BD8DFE803F0070A18
:10F6C0000C41460A0A0A0A0A0A0A3E00A08803F008
:10F6D00009FF02B010BD6088694603F0BBFD08B1A8
:10F6E000FCF77AFE9DF800305B0715D5A08803F083
:10F6F000F9FE03F0CBFD0528EBD9002101AB0DF19C
:10F7000002020846ADF80210019103F0D1FDBDF8E8
:10F71000020003F0C3FDDCE7104C1149208803F020
:10F72000A3FD08B1FCF758FE20881321FFF7E0FD88
:10F730000028CED0FCF750FECBE7FFF7A3FFC8E7C9
:10F74000064B4FF6FF721A80C3E7012360888DF8DD
:10F75000043001A903F07AFDBBE700BF302600208A
:10F7600032260020FCF738BE1F2886BF054A00F06D
:10F770001F004FF0A042012303FA00F0C2F8080571
:10F78000704700BF000300501F2886BF054A00F0E5
:10F790001F004FF0A042012303FA00F0C2F80C054D
:10F7A000704700BF0003005008B50848002240F62B
:10F7B000CD41FCF7F2FE08B1FCF70EFE0C20FFF77E
:10F7C000D3FFBDE808400B20FFF7DEBF203000204C
:10F7D00008B50B48FCF7F9FE08B1FCF7FDFD052064
:10F7E00001F0A2F90C20FFF7CFFF0020FFF77EFD0C
:10F7F000FFF78EFD18B1BDE80840FCF7EDBD08BD70
:10F80000002B0020000000002DE9F041A84BA94E7C
:10F810001A68A94D2DED028B82B0BAB9A74B3260A0
:10F82000A74801221A70FCF7D0FEA64B01220C203B
:10F830001A70FFF7A9FF0B20FFF796FFFCF7D0FE29
:10F84000286002B0BDEC028BBDE8F08193ED007A38
:10F85000DFED9D6A9D4CDFF8C082B8EE477A002745
:10F86000C7EE267A0A20FCEEE77AC4ED007A1F6024
:10F87000FFF77AFF964B4FF47A4043F00103984725
:10F880000DF106013846FFF775FBBDF806309FED18
:10F89000917A4FF4167213FB02F3BB42B8BF03F226
:10F8A000FF3306229B12534307EE903AF8EE677A35
:10F8B000894FC7EE277A17EE900A05F065FA874B55
:10F8C000002205F053F86EA3D3E9002305F052F8A7
:10F8D00005F074FADFED827A07EE100AC7EE277A98
:10F8E00017EE900A05F050FA41EC100B05F0FCFA07
:10F8F00065A3D3E9002351EC100B05F03BF864A39A
:10F90000D3E9002304F010FF02460B4662A1D1E9BF
:10F91000000105F0CBF805F051FA05F035FA60A3C7
:10F92000D3E9002305F022F805F048FA07EE900A23
:10F930000A20FFF729FF9FED6B7A67EE877AFCEECE
:10F94000E77A17EE903A9BB2A8F80030FCF748FE31
:10F950002968FCF740FE3B88C0F3903010FA83F32F
:10F960009BB23B802068E0B105F000FA5E4B0022BC
:10F9700005F09CF84CA3D3E9002304F0D5FE5B4BC3
:10F98000002204F0F7FF5A4B002205F08FF805F033
:10F9900015FA05F0F9F9574B002204F0C5FE05F001
:10F9A000BDF9554C306096ED007AD4ED007AB8EE92
:10F9B000477AF8EE677AB1EE048AE7EE087AFCEE51
:10F9C000E77AC4ED007A20683B889BB2B0FBF3F085
:10F9D00007EE900AF8EE677A17EE900A05F0D4F970
:10F9E000444B002204F0A0FE05F098F9434B444A32
:10F9F0001860D6ED006AB8F80030D2ED007A9BB2FC
:10FA000007EE103AF8EE666AB8EEC77A66EE886AD4
:10FA1000F8EE677AE6EE877AFCEEE77AC2ED007AD6
:10FA200013682268B3FBF2F3364A9BB21380226854
:10FA300041F26F739A4213D9002233484FF40051B8
:10FA4000FCF7ABFD314B01221A70314931480022DD
:10FA5000FCF7A3FD00283FF4E8AEFCF7BDFCE4E6AC
:10FA6000226841F287339A4203D9012001F05CF801
:10FA7000EBE7226840F2DB539A42E6D90420F5E72F
:10FA800000000000000BE3400000006066A272402E
:10FA900000000000009AB04000000080C1553341D2
:10FAA0006666666666127140CDCCCCCCCCCCEC3FA1
:10FAB0001C300020242B0020703000206C300020EF
:10FAC000302B002011300020CDCCCC3D2C2B002041
:10FAD000B0540200000057452A2B00200000F03FE0
:10FAE0000050C3470000C8420080714000408F4072
:10FAF00000004E400000E03FC8300020F82A0020FF
:10FB0000C0300020FC2A0020403000209830002027
:10FB1000CD2C0100502B0020282B00204FF010226C
:10FB20002DE9F047D2F8043303F00703052BB6B0F4
:10FB30001BD01F4B0122C3F80425D3F80024002A50
:10FB4000FBD04FF01021D1F8042322F0070242F03D
:10FB50000502C1F804230022C3F80425144AD2F890
:10FB60000034002BFBD0FFF7AFFBD2F80C7217F07C
:10FB700001071FD00E4B0122C3F80425D3F800243F
:10FB8000002AFBD04FF01022D2F80C3223F00103F0
:10FB9000C2F80C32064B1A46D3F800140029FBD0E9
:10FBA0000021C3F80415D2F80034002BFBD0DAE7AB
:10FBB00000E001400120FFF7ADFBFEF7ABFC08B110
:10FBC000FCF70AFCFEF73CFD002800F09E82AD4BDE
:10FBD000AD4A18689B880B90ADF83030AB4840F6C2
:10FBE000FF730BA9ADF82C30FFF7D2FA08B1FCF780
:10FBF000F3FBA648FFF70EFBFCF792FC08B1FCF7FD
:10FC0000EBFBA34AA3480021FCF7BCFC08B1FCF7BE
:10FC1000E3FBA14AA1480021FCF7B4FC08B1FCF7C2
:10FC2000DBFB9F4A9F480021FCF7ACFC08B1FCF7C6
:10FC3000D3FB9D4A9D480121FCF7A4FC08B1FCF7C9
:10FC4000CBFB9B4A9B480021FCF79CFC08B1FCF7CE
:10FC5000C3FB994A99480021FCF794FC08B1FCF7D2
:10FC6000BBFB974A97480121FCF78CFC08B1FCF7D5
:10FC7000B3FBFEF785F908B1FCF7AEFB04F00CFC12
:10FC800008B1FCF7A9FB00230BA901200B9304F09A
:10FC9000CBFC08B1FCF7A0FB0BA804F01BFD08B1DE
:10FCA000FCF79AFB312388488DF8143005F031FBBE
:10FCB000854982B205A8FFF721FB08B1FCF78CFB50
:10FCC0000020FFF717FB08B1FCF786FB0822002194
:10FCD0000BA805F0EBFA7D4A4FF0C8730BA8CDE9ED
:10FCE0000B23FFF709FB08B1FCF776FB784B79494A
:10FCF00018689A88089008AD9B79ADF824202220D6
:10FD0000AB710D60FFF7FEFA08B1FCF765FB7248B6
:10FD1000002102F056FC08B1FCF75EFB6F4B704807
:10FD20000893294602F002FD08B1FCF755FB0021BB
:10FD300020220BA805F0BAFA6A4B0B9300230C9310
:10FD400043F23113ADF84830674831230BA98DF8E1
:10FD50004A3000F0D5FA08B1FCF73EFBAC22002196
:10FD60000BA805F0A3FA4FF4C062ADF82E200122D3
:10FD700000235E49ADF834208DF8A82041F270725E
:10FD8000CDE92D238DF82C300E91594B59483493E1
:10FD90000BA901F0B9F908B1FCF71EFB5548012188
:10FDA00001F0AFF91C2200210BA805F07FFA002317
:10FDB0004FF4A032CDE90B32ADF83A304FF4F022D7
:10FDC0008DF83C304C4B0D92109303224B4B8DF829
:10FDD00038200BA8119301F04BFC08B1FCF7FCFA9A
:10FDE00003F0D6F908B1FCF7F7FA052200210BA8B9
:10FDF00005F05CFA0B9B03F07C42414B13430B93E1
:10FE00009DF8303023F0030343F003030BA88DF873
:10FE1000303003F003FA08B1FCF7DEFA394803F09A
:10FE2000E5F908B1FCF7D8FA3748FDF7E5FAFDF730
:10FE3000F9FA08B1FCF7D0FA344C2378002B00F023
:10FE40006781122200210BA805F030FA0BA8FDF7FC
:10FE5000CDFC08B1FCF7C0FAFEF77CFC08B1FCF75A
:10FE6000BBFA2B4B1A889B78ADF82020AB70294A3F
:10FE70000023294605208DF82130FEF713FD0028C8
:10FE80004CD049E09254020059F30100D4540200CE
:10FE900009F80100B8540200A9F70100BC5402009F
:10FEA00061F30100C0540200F5F40100AC540200FB
:10FEB000D1F70100DC5402005BF30100E0540200C2
:10FEC000D5F40100D0540200685402005000200311
:10FED0007E54020014300020A82F002089F3010076
:10FEE000C02F002019F30100CC2F00202C26002069
:10FEF00021F50100702B002045F5010065F7010098
:10FF000003071003A1F6010021F30100A52F002033
:10FF10009854020065F50100FCF75EFA0121052006
:10FF2000FEF73CFD4FF0A0434FF40032C3F8142716
:10FF3000974B0BAC1A889B78ADF82C2021460C20EF
:10FF4000A370FEF73FFC08B1FCF746FA0C20FFF760
:10FF50001BFC21460E20FEF735FC08B1FCF73CFAED
:10FF600021460F20FEF72EFC08B1FCF735FA21469A
:10FF70000D20FEF727FC08B1FCF72EFA21460A20D7
:10FF8000FEF720FC08B1FCF727FA0A20FFF7FCFB7C
:10FF900000F07EFD7F4B93E8070041F2883384E850
:10FFA00007007D490C932046FEF730FE08B1FCF7B0
:10FFB00013FA7A48FEF764FE08B1FCF70DFAFEF773
:10FFC00051FE042000F0B0FD0A20FFF7DDFB2046C3
:10FFD000FFF79AF900264FF0FF30FFF797F912224A
:10FFE00031462046CDE90566CDE90166079605F064
:10FFF0005DF92046FDF7FAFB08B1FCF7EDF9DFF8F3
:020000022000DC
:100000009C81DFF8A0910896C5E901660026BDF83D
:1000100030309E427FD3FFF735FB6148DFF8B8915F
:10002000604F00224FF42031FCF7B7FA5E4EFDF727
:10003000D1FF98F80000FEF749FE99F80030002B38
:10004000F5D0FFF717FA3378002BF0D0FFF712FA4C
:10005000FFF764F8554B1B88BB80554B1B88FB8012
:10006000544B1B68BB603B680026642BC5E90066E7
:10007000CDE90366C4E90066AE60A66000F2AE801A
:100080004D4B4E491E703046FDF726FB8246FFF76A
:10009000E7F948F206639A4569D1DFF838A18AF892
:1000A0000060FDF74DFB08B1FCF796F99AF80030B7
:1000B000002B59D0052000F037FD394800224FF4BD
:1000C0002031FCF76AFA08B1FCF786F93C4B1B7843
:1000D00013B13C48FCF779FA3B4B1B7803F0FF0265
:1000E000002B40F0C58039484FF40051FCF755FA19
:1000F00008B1FCF771F9364B00220C201A70FFF79B
:1001000043FB0B20FFF730FB90E7FEF71FFA59E5A2
:10011000FDF760FF91E698F80000FEF7D7FD01219A
:1001200001AB05AA0846FDF731FBD8B9CDE90300BC
:1001300003A905A8FDF786FAA0B904990C22284660
:1001400005F08BF805A8FDF7A3FA08B1FCF744F910
:10015000DDF820A0BA4505D90C222946484605F00D
:100160007CF85746013652E7FDF734FF9EE7BAF1B7
:10017000000F9FD05046FCF72FF99BE7FDF72AFFB1
:100180006CE0FFF76DF9002E94D03046F3E700BF26
:100190009B540200A05402001BF30100A42F002076
:1001A00078300020603000206C300020FC2A0020D5
:1001B0002A2B0020C830002010300020C454020038
:1001C0009830002040300020202B0020002B002001
:1001D00074300020BC2F002011300020012103AB1F
:1001E00008AA0846FDF7D2FA064600287FF462AF57
:1001F00098F80000FEF76AFD05A908A8CDE9056694
:10020000FDF720FA20B906990C22204605F025F8C2
:1002100008A8FDF73DFA08B1FCF7DEF80B9A38683C
:100220006423B2FBF3F103FB1121B0FBF3F203FBF8
:1002300012039942D2D1124B12494FF0000A08A87A
:1002400083F800A0FDF74CFA48F206639842064690
:1002500097D10D4E86F800A0FDF772FA3378002B87
:100260008CD0084908A8FDF73BFAFFF7F9F821E719
:10027000032000F059FC054800224FF4203135E7F7
:1002800010300020C4540200BC2F0020A0300020F9
:10029000A8DF7047AADF7047ACDF7047AEDF70475A
:1002A00062DF704713B50C4681B178B10388112B1A
:1002B0000ED0502B11D0102B08D18388CB8703236D
:1002C0008DF80430236801A92046984702B010BD7C
:1002D0004FF6FF73CB870223F2E7C2884B8C9A421A
:1002E000F4D1038A022BF1D10B68002BEED012302F
:1002F00001F05AFB80F001008DF80400E2E70000F5
:100300002DE9F04F0D4695B00646002800F06182B9
:10031000002900F05E820B6803604FF6FF73C3870D
:10032000CD4B04AA03F1100C1746186859681446FF
:1003300003C4083363452246F7D106F1400138462D
:10034000FFF7AEFF0446002840F0448296F84030A4
:100350008DF80A30321D4FF4A05302A90120ADF8E8
:100360000830FFF795FF0446002840F0338201462D
:100370000322684604F09AFF2B7F8DF801309DF828
:1003800002304FF0010969F342031C2221464FF06D
:10039000110A0DA88DF802308DF800A004F086FF38
:1003A0009DF83430119423F01A0343F012038DF8B2
:1003B0003430AA4B0E934FF01213CDE90F3401AF36
:1003C00096F840308DF80E30032241F20143214669
:1003D0003846ADF80C30CDF848D0139404F066FFE1
:1003E0006B7F8DF80430AB7F8DF805309DF80630BB
:1003F00023F01F0343F002031422214608A84FF004
:10040000040B8DF8063004F051FF03ABCDE908373B
:1004100005EB0B030C93B088CDF828B0B31D08AAE8
:100420000DA9ADF82CB0FFF735FF002840F0D181C1
:1004300003222146684604F039FF2B7F8DF80130F6
:100440009DF802308DF800A069F342031C2221467A
:100450000DA88DF8023004F029FF9DF83430119476
:1004600023F01A0343F012038DF834307C4B0E93C3
:100470004FF02B13CDE90F3496F840308DF80E3045
:10048000032241F2024321463846ADF80C30CDF844
:1004900048D0139404F00AFF6B7F8DF80430AB7FD3
:1004A0008DF805309DF8063023F01F0343F002035A
:1004B0001422214608A88DF8063004F0F7FE03AB9D
:1004C000CDE9083705F108034FF002080C93B08816
:1004D000CDF8288006F10E0308AA0DA9ADF82C80EE
:1004E000FFF7D8FE002840F07481032221466846B9
:1004F00004F0DCFE2B7F8DF801309DF802308DF882
:1005000000A069F342031C2221460DA88DF8023099
:1005100004F0CCFE9DF83430119423F01A0343F01C
:1005200012038DF834304F4B0E934FF03013CDE95A
:100530000F3496F840308DF80E30032241F2034319
:1005400021463846ADF80C30CDF848D0139404F06D
:10055000ADFE6B7F8DF80430AB7F8DF805309DF8D4
:10056000063023F01F0343EA08031422214608A89B
:100570008DF8063004F09AFE03ABCDE9083705F19B
:100580000A030C93B088CDF8288006F1160308AA58
:100590000DA9ADF82C80FFF77DFE002840F01981F1
:1005A00003222146684604F081FE2B7F8DF801303E
:1005B0009DF802308DF800A069F342031C22214609
:1005C0000DA88DF8023004F071FE9DF834301194BE
:1005D00023F01A0343F012038DF83430224B0E93AC
:1005E0004FF02A13CDE90F3496F840308DF80E30D5
:1005F000032241F2044321463846ADF80C30CDF8D1
:1006000048D0139404F052FE6B7F8DF80430AB7F1A
:100610008DF805309DF8063023F01F0343EA0803E8
:100620001422214608A88DF8063004F03FFE03ABE3
:10063000CDE9083705F10C030C93B088CDF828B04C
:1006400006F11E0308AA0DA9ADF82CB0FFF722FE93
:10065000002840F0BE8009E0E4540200B6260020E5
:100660006426002034260020C826002003222146CC
:10067000684604F01BFE2B7F8DF801309DF8023098
:100680008DF800A069F342031C2221460DA88DF8C5
:10069000023004F00BFE9DF83430119423F01A035D
:1006A00043F012038DF834304C4B0E934FF030135F
:1006B000CDE90F3496F840308DF80E30032241F228
:1006C000054321463846ADF80C30CDF848D0139498
:1006D00004F0ECFD6B7F8DF80430AB7F8DF80530B6
:1006E0009DF8063023F01F0343EA08031422214635
:1006F00008A88DF8063004F0D9FD03ABCDE9083722
:1007000005F110030C93B088CDF828B006F126034C
:1007100008AA0DA9ADF82CB0FFF7BCFD002858D1F0
:1007200021460322684604F0C1FD2B7F8DF801307D
:100730009DF802308DF800A069F3420321461C2287
:100740000DA88DF8023004F0B1FD9DF834301194FD
:1007500023F01A0343F012038DF83430204B0E932C
:100760004FF02713CDE90F3496F840308DF80E3056
:10077000214641F20643032238461394ADF80C306B
:10078000CDF848D004F092FD6B7F8DF80430AB7F3C
:100790008DF805309DF8063023F01F0343EA080367
:1007A0002146142208A88DF8063004F07FFD03AB23
:1007B000CDE90837B088CDF82880143506F12E032E
:1007C00008AA0DA9ADF82C800C95FFF763FD04462F
:1007D00000B10E24204615B0BDE8F08FF2260020AF
:1007E0008F26002030B589B00446019168B302AD70
:1007F00008220021284604F059FD04230293E188D1
:10080000E08F6B442A460393FFF746FDD8B9E28F89
:100810004FF6FF739A4216D0102201460DEB0200EC
:1008200004F044FDE388ADF8103001238DF8123058
:10083000BDF80A30ADF81430E08F039B069504A98B
:100840000793FFF72BFD09B030BD0E20FBE730B555
:1008500089B00446ADF8061070B302AD082200213D
:10086000284604F023FD02230293E189E08F0DF175
:1008700006032A460393FFF70FFDD8B9E28F4FF620
:10088000FF739A4216D0102201460DEB020004F0CD
:100890000DFDE389ADF8103001238DF81230BDF85D
:1008A0000A30ADF81430E08F039B069504A9079336
:1008B000FFF7F4FC09B030BD0E20FBE730B589B07E
:1008C0000446ADF8061070B302AD08220021284698
:1008D00004F0ECFC02230293E18AE08F0DF10603A1
:1008E0002A460393FFF7D8FCD8B9E28F4FF6FF737F
:1008F0009A4216D0102201460DEB020004F0D6FCFD
:10090000E38AADF8103001238DF81230BDF80A30BB
:10091000ADF81430E08F039B069504A90793FFF709
:10092000BDFC09B030BD0E20FBE730B589B00446F0
:10093000019168B302AD08220021284604F0B6FCFC
:1009400004230293E18BE08F6B442A460393FFF765
:10095000A3FCD8B9E28F4FF6FF739A4216D010224B
:1009600001460DEB020004F0A1FCE38BADF8103062
:1009700001238DF81230BDF80A30ADF81430E08F45
:10098000039B069504A90793FFF788FC09B030BDC7
:100990000E20FBE730B589B00446019168B302AD83
:1009A00008220021284604F081FC04230293E18CF4
:1009B000E08F6B442A460393FFF76EFCD8B9E28FB1
:1009C0004FF6FF739A4216D0102201460DEB02003B
:1009D00004F06CFCE38CADF8103001238DF812307C
:1009E000BDF80A30ADF81430E08F039B069504A9DA
:1009F0000793FFF753FC09B030BD0E20FBE730B57D
:100A000089B00446ADF8061070B302AD082200218B
:100A1000284604F04BFC02230293E18DE08F0DF198
:100A200006032A460393FFF737FCD8B9E28F4FF647
:100A3000FF739A4216D0102201460DEB020004F01B
:100A400035FCE38DADF8103001238DF81230BDF880
:100A50000A30ADF81430E08F039B069504A9079384
:100A6000FFF71CFC09B030BD0E20FBE71F2886BF36
:100A7000054A00F01F004FF0A042012303FA00F0E6
:100A8000C2F80805704700BF00030050704700001F
:100A90001FB54FF4804302931C4B03934FF4C8449B
:100AA0004FF0A0431A4A1B48ADF800406946019335
:100AB000FDF7AAFB08B1FBF78FFC4FF4004302934C
:100AC000154B0393124A1548ADF800404FF0A04370
:100AD00069460193FDF798FB08B1FBF77DFC4FF4E5
:100AE000C843ADF800304FF4005302930C4B03930E
:100AF000074A0C484FF0A04369460193FDF784FB79
:100B000008B1FBF769FC04B010BD00BF0855020036
:100B10008D0A0200783100200C550200F0300020D0
:100B200010550200CC30002070B504462948FDF76E
:100B3000B1FB08B1FBF750FC2748FDF7ABFB08B150
:100B4000FBF74AFC2548FDF7A5FB08B1FBF744FC81
:100B5000042C33D8224D1F4804EB44036600E95CA3
:100B6000FDF7A7FB08B1FBF737FC33192B441A48F4
:100B70005978FDF79EFB08B1FBF72EFC3444254461
:100B80001648A978FDF795FB08B1FBF725FC11483D
:100B90008168FDF76BFB08B1FBF71EFC0E4881680E
:100BA000FDF764FB08B1FBF717FC0C488168FDF703
:100BB0005DFB70B1BDE87040FBF70EBC0E20FFF787
:100BC00055FF0F20FFF752FFBDE870400D20FFF7E3
:100BD0004DBF70BD78310020F0300020CC300020B7
:100BE000F45402006DDF704779DF70477DDF704796
:100BF00064DF70472DE9F04F85B000250E9CBDF8ED
:100C00003CB0B4F800A00191074690461E46A946A4
:100C10003A884A450DDC45B12388013BA3EB0A0322
:100C20009BB2FF2B3AD806F80A30002005B0BDE889
:100C3000F08F7A6852F82900039000220DF10B0121
:100C400003A8FFF7D5FF0028F0D19DF80B204245FF
:100C500021D12288002D14BF0020022002EB0801C0
:100C6000014459451ADC3DB9013292B2019B228000
:100C7000B35422880132228022880DF10B013244C4
:100C800003A8FFF7B5FF0028D0D121889DF80B20DD
:100C90000A442280012509F10109B9E70C20C5E7C2
:100CA0002DE9F341089FBDF824801546CDE9007871
:100CB000022204461E46FFF79DFF50B9334610221C
:100CC00029462046CDE9087802B0BDE8F041FFF79B
:100CD00091BF02B0BDE8F0812DE9F04F00231788E5
:100CE000138090F82D3085B006460D46144653B358
:100CF000082F01D80C2027E102A8FFF773FF002876
:100D000040F0228123880822EA54238801339BB2D1
:100D10001B222380EA542088013080B220800622E2
:100D20000DF10901284404F098FA23889DF8082061
:100D300006339BB212F0FE0218BF01222380EA5450
:100D4000238801332380B378FBB123880433BB426B
:100D5000D0D802A8FFF748FF002840F0F58023888C
:100D60000322EA54238801339BB219222380EA54D8
:100D70002388BDF8082001339BB2E9182380EA5488
:100D8000120A4A70238802332380F2789AB12388AA
:100D9000D91CB942AED80221E954238801339BB251
:100DA00001212380E95423880B449BB22380EA5419
:100DB00023880B4423807268AAB12388D91CB942C6
:100DC00098D8022192F90020E954238801339BB27C
:100DD0000A212380E954238801339BB22380EA54FB
:100DE0002388013323803389002B40F0A180338A8C
:100DF0005BB1CDE900472B460722032106F1100025
:100E0000FFF74EFF002840F09F80338B5BB1CDE9A8
:100E100000472B461522142106F11800FFF740FF6A
:100E2000002840F09180326A002A40F09080D6F885
:100E30002480B8F1000F30D0B8F804302188981C15
:100E40008A1C0244BA423FF655AFFE283FF652AF25
:100E500003336B54238801339BB2FF222380EA546F
:100E6000238801339BB22380B8F80020EA54E918A4
:100E7000120A4A702088023080B22080B8F804201C
:100E80005AB1D8F8081000296BD0284404F0E5F9CD
:100E90002388B8F804201344238096F82C30002BC4
:100EA00040F09A80307800284ED03388012B58D0FB
:100EB000228802F1020CBC453FF61CAF012805D187
:100EC0007378023313449F42FFF414AF023FBF1AFA
:100ED000BFB202A905EB0C00ADF80870FFF786FE63
:100EE00090BB3178BDF80830022900F0BA807278E2
:100EF0009A4202D3BB4240F2B280012940F0B38053
:100F0000974293B2C0F0AF80ADF808300821BDF829
:100F10000830FE2B3FF6EEAE22880133AB54228818
:100F2000013292B22280A9542288134423800BE01C
:100F3000CDE900472B460622022106F10800FFF703
:100F4000AFFE00283FF453AF05B0BDE8F08FB4F812
:100F500000C00CF10603BB423FF6CCAE1188052958
:100F600001D80720F0E76FF4486E01EB0E039BB247
:100F70004FF27D3E7345F4D95388052BF1D96FF4B8
:100F80004860181880B27045EBD94FF6FF70814267
:100F900003D0834201D09942E3D8052305F80C30F1
:100FA000238801339BB212212380E9542388013323
:100FB0009BB223801188E954E818090A41702388FC
:100FC00002339BB223805288EA54E918120A4A700D
:100FD0002388023323802AE7B36A002BC1D04FF065
:100FE00000094FF00C0A4FF0160B96F82C305FFA00
:100FF00089F293427FF656AFB16A0AFB02F201EB27
:101000000208B8F80430981CFE283FF673AE20881A
:1010100003332B54238801339BB2238005F803B09C
:10102000238801339BB223808A5AEA54E918120AB2
:101030004A702088023080B22080B8F804205AB16B
:10104000D8F8081000298CD0284404F006F9238829
:10105000B8F804201344238009F10109C5E70921E8
:1010600055E7BB42FBD9ADF808704FE770B5E8B162
:101070004AB116880024B44203D305196D789D4205
:1010800008D0A14201D8002010E0055D01352C44B4
:10109000A4B2F0E7A142F6D9005D0138A31C80B2EA
:1010A0009DB210FA83F38B42EDDC158070BD13B551
:1010B00013460022ADF806200DF106020446FFF7A4
:1010C000D5FF10B1BDF80630E01802B010BD72DFD8
:1010D000704773DF704738B5012204460D46B0F8FB
:1010E0001414D0F81004FFF7E2FF00B1057004F10A
:1010F0003C0204F5826104F15400BDE83840FFF77A
:10110000E6BF80F830107047F8B504460F46002956
:1011100075D0002873D091F87A301BB191F89830CF
:10112000002B6ED1D7F8A030042B6AD0D7F89C30B2
:10113000042B66D04FF0000C84F802C007F178064B
:101140000FCE251D0FC50FCE0FC596E8070085E809
:10115000070084F830C0D7F8A4306363D7F8A8300C
:10116000A3634FF6FF7504F58263C4F82034A4F836
:1011700024540722614604F2264004F097F82378AD
:101180000BB984F8545094F82430002B14BFEE238C
:101190001F2304F15501C4F81014A4F8143404F208
:1011A00014423846FFF798FD40BB94F82430002BDA
:1011B00014BFEE231F2304F23121C4F81814A4F83D
:1011C0001C3404F21C4207F13C00FFF785FDA8B96E
:1011D000A369A4F848304FF480730125A4F8503077
:1011E00063692064014684F83C50636404F13C0266
:1011F00004F15400FFF76BFF00B92570F8BD0E2015
:10120000FCE70720FAE7F8B5077804460D46002FFB
:1012100000F0F88000F22646817007220021304657
:1012200004F044F8E38813B1A378012B04D0E379E8
:101230004BB1A378022B06D1636BA3B1012284F8D2
:101240002D2408209847334604F22C4113F8012F2F
:1012500012B99942FAD117466B1E032B51D8DFE819
:1012600003F0050B0F1284F82D34ECE7A3791BB1C2
:1012700094F8243003B95FB9E3790BB1002F42D160
:10128000237A002B41D1637A002B0CBF0025042563
:10129000636BA570002B3AD0033D012D37D86279DE
:1012A000AAB394F82E2492BB84F83024012284F847
:1012B0002F240720984704F13C05182200212846D6
:1012C00003F0F4FFE26A531E0121022B94F824304C
:1012D00084F83C1028BF0A4684F8512033B1A36A31
:1012E0005A1E022A28BF0B4684F85230A2780023E7
:1012F00084F85030042A1BD8DFE802F06C0D22324B
:1013000052000025C4E70225C2E70325C0E70023F9
:1013100084F82F34CFE7C4E91063C4F820340223E3
:10132000012284F83C30802384F83120A4F848302E
:10133000A378002B51D1636B002B5FD100205CE0C0
:10134000022384F83130032384F83C302369A4F865
:1013500048300023C4F82034E36826646364E7E778
:1013600063696364A369A4F848306379B3B194F8FE
:101370002E349BB994F8303483B1022384F8503072
:1013800004212046FFF7A7FE0028D1D1052384F8C9
:10139000313004F58263C4F82034C9E70323F6E74B
:1013A000E3696364236AA4F84830637983B194F8ED
:1013B0002E346BB994F8303453B1022384F8503092
:1013C00004212046FFF787FE0028B1D10623DEE77F
:1013D0000423DCE784F83130AAE7D4F820142A4645
:1013E00004F15400FFF773FE38B994F8301094F804
:1013F0005400FFF76EFE00289DD0F8BD94F8310030
:1014000098479BE70820F8E70388112B10B50C4696
:101410000AD0262B1FD0102B05D1C37B012B02D164
:101420008388A1F8243410BD0022838881F82E24FB
:10143000B1F824249A42F6D10B79002BF3D1012183
:101440002046FFF7E0FE0028EDD0A36B002BEAD08A
:10145000BDE810401847037A013B012BE3D8897897
:1014600005230131B1FBF3F303EB8303C91AC9B2BE
:10147000E6E775DF704776DF70477ADF70477BDF1E
:1014800070470000034B1A8882420CBF18460020A8
:10149000704700BFB8310020024B9B6903B1184769
:1014A000704700BF9C31002073B585B22846FFF716
:1014B000E9FF044670B1164E027A337B9A420BD292
:1014C00000F10A012846FFF7D4FFE8B1112801D046
:1014D000FFF7E2FF02B070BD00230372337C43B11B
:1014E0003B212846FFF7C7FF30F0080301D0FFF784
:1014F000D3FF7369002BEDD000228DF80420ADF8E6
:10150000065001A89847E5E7237A01332372E1E703
:101510009C31002037B50B46497A0F4A71B9D2E9A0
:1015200001141D7A0246002D18BF21465868FBF7AA
:1015300034F808B1FFF7B0FF03B030BD00211972D5
:101540005369002BF8D00122ADF806008DF8042075
:1015500001A89847F0E700BF9C3100204B88028823
:101560009A4213D842889A4210D380888A8840F2DF
:10157000F313984294BF031AC31A934206D800F299
:10158000F310904234BF00200120704700207047C4
:101590000388122B70B5014659D004D8102B1ED0E9
:1015A000112B44D070BD502BFCD12F4BC288DB894E
:1015B0009A42F7D1038A022BF4D186883046FFF78E
:1015C00061FF05460028EDD001F1120000F0ECF9B2
:1015D00038BB6868FAF7F9FF0028E3D009E0C37B5D
:1015E000012BDFD14FF6FF70FFF74CFF054620B906
:1015F0000420BDE87040FFF74FBF1C4A8E8806806C
:10160000002303721368C0F80A305368C0F80E3024
:1016100010310A30FFF7A2FF134B6872DB89002BF1
:10162000C0D129463046BDE87040FFF773BF8088BF
:10163000FFF728FF04460028B4D04068FAF7C5FF3A
:1016400008B1FFF729FF4FF6FF732380AAE78688CA
:101650003046FFF717FF05460028A3D008310A30AF
:10166000FFF77CFF6872DCE79C310020CC31002062
:10167000F8B5064648B305460FCD154F3C460FC496
:1016800095E8070084E807003068124C3C60B0B170
:10169000FFF7F3FEC0B932681368236053686360D4
:1016A0000D480E4A4FF6FF7303800D4B40F8043F80
:1016B0000021FAF767FF002818BF032004E0204646
:1016C000FFF7DDFE0028EBD0F8BD0E20FCE700BFE1
:1016D0009C310020CC310020B8310020A914020038
:1016E000D8310020F7B5174601900E4691B1019C04
:1016F0006CB100252C46294601A8FCF7C4F918B1A5
:101700003946A8B2B04701340135142DF3D1204633
:1017100003B0F0BD0C46FAE70AB1FCF793B9FCF749
:10172000A8B973B50191019C06466CB100252C4601
:10173000294601A8FCF7A7F918B106EB44030134C8
:101740009D800135142DF3D13046346002B070BD58
:101750002DE9F04703888488103B8CB005460A2B9E
:101760001FD8DFE803F0063F1E1E1E1E1E1E1E6051
:101770004400314EB368DB43009371686846FCF760
:10178000DBF9009901A8FFF7CCFF0DF108094FF034
:101790000008019B984507D3132C13D90420FAF7AE
:1017A0001BFE0CB0BDE8F08739F802AB002701370B
:1017B000514606EB8700FCF75CF91E2FF7D108F1C4
:1017C0000108E6E71D482146FCF73CF91C48214684
:1017D000FCF738F9EB7B012BE3D01A482146FCF7E4
:1017E00031F9DEE715482146FCF743F9D9E7027ADB
:1017F00015483F2A4FEA1215214694BF00220122C4
:10180000FFF78AFF022D94BF002201220F482146D4
:10181000FFF782FF012D0E4894BF002201222146CE
:10182000FFF77AFFBDE7037A002BBAD1427A064868
:10183000C2F3C0022146F3E7F83100200032002055
:10184000FC31002004320020103200200C32002035
:10185000083200201328014602D80248FCF713B9C9
:1018600000207047FC310020FFF7F4BF07B501905E
:10187000FFF7F0FF019930B10448FCF704F90028A4
:1018800014BF0220012003B05DF804FB00320020E9
:1018900007B50190FFF7DEFF019928B1044803B0B6
:1018A0005DF804EBFCF7EFB803B05DF804FB00BF94
:1018B0000832002007B50190FFF7CCFF019928B14D
:1018C000044803B05DF804EBFCF7DDB803B05DF845
:1018D00004FB00BF0C32002007B50190FFF7BAFFF0
:1018E000019928B1044803B05DF804EBFCF7CBB8CC
:1018F00003B05DF804FB00BF1032002008B51821CA
:101900000248FCF7C9F8C0B208BD00BFF83100209A
:1019100070B50A4E054630460C46FCF7B4F858B18F
:101920002846FFF797FF38B10734294606EB8400B5
:10193000BDE87040FCF7A7B8002070BDF83100206A
:10194000F8B50B4F054638460C461646FCF79BF893
:1019500060B12846FFF77EFF40B107343246294682
:1019600007EB8400BDE8F840FFF7D6BEF8BD00BF26
:10197000F831002073B50B4D019204460E46014626
:101980002846FCF780F850B1063405EB8404019A30
:101990006068314602B0BDE87040FFF7A3BE02B0F8
:1019A00070BD00BFF8310020007800F001007047E2
:1019B000A0DF7047A1DF7047ADDF7047B3DF70472E
:1019C000B4DF704710B50446408800F07DFCA0806D
:1019D0002046BDE8104001F0D5BB30B587B00546C4
:1019E0000C461422002101A803F060FC072301A883
:1019F0008DF80430ADF806500394FFF7E3FF07B00D
:101A000030BD000030B587B005461422002101A882
:101A100003F04CFC4FF6FF739D42ADF8065023D007
:101A2000284600F064FB1128044617D007D860B19F
:101A30000B2811D021462846FFF7CFFF03E043F2E1
:101A400002039842F6D1002209E00E2301A88DF886
:101A50000430FFF7B7FFF6E70F23F7E70122034B48
:101A600028461978FFF76CFF07B030BD7B320020A5
:101A7000FFF7C8BF024B034918780022FFF77ABF6F
:101A80007D320020891A02002DE9F0473E4C88B0D3
:101A900021780546FFF73CFFA046064600286CD19A
:101AA000284600F077FB0828014622D006D888B1E6
:101AB00006284BD02846FFF790FF09E043F20203C7
:101AC000984205D043F20143984259D01128F1D1F0
:101AD000012446E03146142203A803F0E7FB10235B
:101AE00003A88DF80C30ADF80E500126FFF76AFF01
:101AF000EEE70DF10600FFF761FF344601274FF0D6
:101B0000020A0DF10809BDF80630BB421ED90022B9
:101B100049463846CDE903A9FFF752FFB0B9BDF8F1
:101B200008303CB942F605241B1B5C425C4101377E
:101B3000BFB2E8E742F602129342F8D101AB03AA22
:101B4000394628460493FFF737FF30B1284600F0A6
:101B5000BBFB00F039FB002403E0BDF80430002B90
:101B6000F4D00A4B224619782846FFF7E9FE98F888
:101B7000001032462846FFF7E3FE08B0BDE8F087C4
:101B80002846FFF73FFFA3E77E3200207D3200208A
:101B900013B5044600F098FB00236A46092100F0C3
:101BA0003FFF052805D1044B012219782046FFF795
:101BB000C7FE02B010BD00BF7932002008B5084B47
:101BC000084918780022FFF7D5FE024630B9064BC7
:101BD00006491878BDE80840FFF7CCBE08BD00BF35
:101BE0007C320020391C020079320020F11B0200F7
:101BF00037B5044604220021684603F057FB42F63D
:101C0000A623ADF800300A4B18680190012501AAFF
:101C1000694620468DF80250FFF7CAFE28B9054BE9
:101C20002A4619782046FFF78BFE03B030BD00BF6F
:101C3000145502007832002030B5012187B00546E6
:101C40001C48FBF756FF0446BFF35F8F70BB284666
:101C500000F008FA862801460ED007D8D0B1112826
:101C600026D02846FFF7B9FE002403E043F2020322
:101C70009842F6D122460FE01422214601A803F033
:101C800015FB062301A88DF80430ADF80650FFF7C8
:101C900099FEEFE701240246074B28461978FFF723
:101CA0004FFE1CB9BFF35F8F024B1C6007B030BD05
:101CB0000122F1E7743200207C32002038B503782D
:101CC0000446A3B94088FFF79DFE6588284600F0CA
:101CD0004EFA28B1064B012219782846FFF730FE4C
:101CE0006088FFF755FFBDE83840FFF767BF38BD94
:101CF0007D32002037B50378082B044630D1427A74
:101D000072BB057A072D1BD0082D2DD0012D27D1B0
:101D100080886A46294601F0B1F808BB019B1B7810
:101D2000F3B1A08800F0FEFA4FF6FF73984217D087
:101D3000114B2A461978FFF703FEFFF79BFE0FE0D1
:101D4000808800F0EFFA4FF6FF739842044607D000
:101D50000A4B01221978FFF7F3FD2046FFF718FF21
:101D6000FFF72CFF03B030BD054B19680129F7D1EF
:101D7000BFF35F8F1A60F3E77D3200207C320020D2
:101D8000743200202DE9F843FFF7B8FDDFF890909A
:101D9000DFF8908089F80000FFF7B0FD88F80000B8
:101DA000FFF7ACFD184F194E3870FFF7A7FD3070E4
:101DB000FFF7A4FD164D174C2870FFF79FFD20700C
:101DC000FFF79CFD144B187099F80030182B18D0B1
:101DD00098F80030182B14D03B78182B11D033789A
:101DE000182B0ED02B78182B0BD02378182B08D05B
:101DF000182806D0094B00201860BFF35F8FBDE89C
:101E0000F8830320FBE700BF7D3200207E320020F4
:101E100079320020783200207A320020743200209B
:101E20007C3200207B32002073B50123ADF80030F6
:101E300009238DF802300D4B002422460E461978F6
:101E4000CDF8034005468DF80740FFF779FD084BB4
:101E500008492846A64218BF1946019100F034FAF5
:101E60002246694600F048FE02B070BD793200207B
:101E70001C5502001855020070B503888488502B49
:101E800086B0054637D00DD8352B47D0362B62D0DB
:101E90003E4B3F4918780022FFF76CFDFFF7EAFD43
:101EA00006B070BD522B22D0542BF1D11422002148
:101EB00001A803F0FBF9112320468DF80430ADF89A
:101EC000064000F001FAADF8080000F07DF9314B52
:101ED000204619780022FFF733FD2F4B2046197852
:101EE0000022FFF72DFD01A8FFF76CFDD0E720468B
:101EF000FFF788FDCCE7037B012BC9D1827A012A49
:101F0000C6D1018942F602139942C1D1234B204622
:101F10001978FFF715FDFFF751FEB9E7204E20466F
:101F20003178FFF7F5FC0028B2D000223178204646
:101F3000FFF706FDEA883ABBAE89012E24D1E98974
:101F40002046FFF737FDF8B9164B32461978204680
:101F5000FFF7F6FC9CE7134E20463178FFF7D8FCDC
:101F6000002895D0317800222046FFF7E9FCE98867
:101F700051B9EB89012B03D1297C003918BF01210C
:101F80002046FFF751FF83E70021F9E77B3200206D
:101F9000711A02007E3200207D3200207C32002047
:101FA000783200207A320020AFDF7047B1DF70470F
:101FB000B2DF7047B3DF704710B50446808800F089
:101FC000B1F960802046BDE8104001F0DDB80000A6
:101FD000F0B5184B184D93E8030089B001AE86E8C0
:101FE00003004FF6FF772888B8421CD00022314604
:101FF00000F082FD0446C0B11422002103A803F0C2
:1020000055F92B88ADF81030112C0CD0862C0CBF54
:102010000623072303A80EBF8DF80C308DF80C3073
:102020000594FFF7C9FF09B0F0BD288800F0BEFD98
:102030002880D8E72055020080320020044B1A88FF
:102040004FF6FF739A4201D0FFF7C2BF704700BF3F
:1020500080320020024B4FF6FF721A80002070473A
:10206000803200202DE9F743804600F02DF94FF62D
:10207000FF739842064637D001274FF003093A46CE
:102080006B460821304600F0FDFE0137BFB2054621
:1020900028BB01990A46032342F8049B06314046B7
:1020A000FFF786FF044648B932460821304600F063
:1020B00072FF0446204603B0BDE8F0830C280CD024
:1020C000052800D12C460821304600F03BFF0028AF
:1020D00018BF0324002DD2D1ECE70125F3E7072830
:1020E00014BF04460C24E5E743F20204E2E72DE9BD
:1020F000F341074600F0E8F84FF6FF73984218D115
:102100000024032526464FF001082B46224631467F
:102110003846FFF74BFF042821D0082825D00B288C
:102120001ED115F002030FD196B9ACB902B0BDE8CB
:10213000F0816A46082100F0A1FE0028E0D1019B51
:102140009C881D689E1DDEE701254FF00008DCE736
:1021500003251C461E46F8E703253446F5E7112003
:10216000B8F1000F08BF0B20E0E70020F8E71FB52B
:102170000DF10703039300F0A7F802AA012100F074
:102180007DFE20B9039B187805B05DF804FB0020A4
:10219000FAE7000070B505460A48FFF70BFF70B973
:1021A000084C43F2030621884FF6FF722846FFF7DA
:1021B000FBFEB04204D1238801332380F3E70320E0
:1021C00070BD00BF8232002013B5074A044692E872
:1021D00003006B4683E8030000221946204600F006
:1021E0008BFC02B010BD00BF2855020046DF7047CF
:1021F000421E00F10F0312F8010F10B99A42FAD1F2
:1022000070470120704708B570B171B103780A7842
:10221000534013F0FE0F08D106220131013002F0C5
:10222000E9FFB0FA80F0400908BD0020FCE72DE985
:10223000F04700F101084F1C06460D4600F1110958
:1022400001F1110A10223946404602F0D3FF04463C
:10225000D0B94046FFF7CCFF18B13846FFF7C8FFAA
:10226000044651464846FFF7CEFF737C03F0FC035B
:10227000042B05D06B7C03F0FC03042B18BF044631
:1022800004F00100BDE8F0870024EAE730B585B02E
:1022900004460D4600F0FAFB02AA0DF106010720E4
:1022A00000F0FCFB10B94FF6FF700BE0BDF80630F4
:1022B000AB42F1D003992046FFF7B9FF0028EBD0DD
:1022C000BDF8060005B030BD132810B5044602D98C
:1022D0004FF6FF7010BDFFF7BDFA0028F8D00A20B6
:1022E000014B4443185BF5E784320020132838B5CE
:1022F00004460D4602D943F2020038BDFFF7AAFAA0
:102300000028F8D006480A2303FB040050F8023FD7
:102310002B608388AB808379AB710020EDE700BF31
:10232000843200204FF6FF7398422DE9F0410546B4
:102330000CD00C4F00244FF00A0808FB04F3A6B29F
:10234000DB5BAB4205D00134142CF6D14FF6FF769F
:1023500004E03046FFF77EFA0028F4D03046BDE8AE
:10236000F08100BF84320020038843B9821C00F151
:102370000A0312F8010B10B99A42FAD170470120F2
:10238000704710B50446FFF7EFFF58B122880B885D
:102390009A4208D108220231A01C02F02BFFB0FAA9
:1023A00080F0400910BD0020FCE71FB5044600F096
:1023B0006DFB02AA0DF10601072000F06FFB10B9BA
:1023C0004FF6FF7007E0039920464631FFF7D9FF2B
:1023D00018B1BDF8060004B010BD039920462A319B
:1023E000FFF7CFFF0028E4D0F3E7000013289FBFDA
:1023F0000A235843014B1952704700BF8432002012
:1024000038B50546FFF78EFF0446284600F0A4FDC8
:1024100038B9132C05D80A235C43024B4FF6FF72E0
:102420001A5338BD8432002070B58CB014466A4609
:102430000D4600F11003164613F8011D02F8011BAA
:102440009842F9D10D22002104A802F02FFF2B7829
:102450008DF81F306B788DF81E303046AB788DF8D4
:102460001D30FFF7C3FE9DF82F3023709DF82E30EE
:1024700063709DF82D30A3700CB070BD30B503783B
:1024800003F0FE03042B85B004460D4618D1411C11
:10249000032201A802F0E1FE0322211D03A802F09D
:1024A000DCFE02AA03A92846FFF7BEFF032202A909
:1024B00001A802F09FFEB0FA80F0400905B030BDDF
:1024C0000020FBE730B50388102B93B04ED1041DDC
:1024D0000FCC07AD0FC50FCC0FC594E807009DF8D2
:1024E000203003F0FE03062B85E8070009D000F03A
:1024F000CDFA9DF82030032B4FEA530204D9022A6B
:102500003DD04FF6FF7310E002AA0DF1060107203F
:1025100000F0C4FA0028F4D0039908A81131FFF79D
:1025200072FE0028F0D0BDF80630BDF81C401848F7
:102530000A226243811883529DF8262008980A7265
:102540004FF6FF72C1F802009342BDF82400C88024
:102550000CD0ADF80C3002A80023ADF80A408DF87D
:10256000083000F013FE02A8FFF7A8FB13B030BD3F
:10257000039908A80131FFF781FF0028D3D102AAEF
:102580000DF10601072000F089FA0028F0D1B8E724
:102590008432002090DF7047A5DF7047B5DF7047B9
:1025A0001FB50023ADF80810ADF80A106A4602A95D
:1025B00003930093ADF80430FFF7ECFF05B05DF82E
:1025C00004FB78B14FF0171303601B23037117232B
:1025D000C380038141F61B32002301614381828164
:1025E000184670470E20704713B5034680880C4686
:1025F00098B91A88242A70D011D8112A4DD0232ACC
:1026000078D0102A2BD0A37A3BB1E1880020FFF7C5
:10261000C3FF10B94FF48073638102B010BD3A2A32
:1026200043D0552AEFD1DB88C988A072172B38BF59
:1026300017238B4228BF0B462381FFF7AFFFE37AB6
:10264000002BE0D12369002BDDD040F677220092E9
:102650002289ADF80420694620469847D3E7DB7B02
:102660000A790A73012B04BF0B88CB80C9882389A0
:102670008B4205D20020FFF78FFF48B90123E37298
:10268000217B637B8B42BED20020FFF789FFBAE734
:10269000112804BF0123A372F2E71723CB800B811B
:1026A00041F61B3348818B81ADE75B89CA88934231
:1026B00028BF1346172B0A6938BF17230B814AB16D
:1026C000C97A39B140F677210091ADF804306946F6
:1026D000204690470023638195E71A7A0B694A7375
:1026E000002B90D04DF67A218DF8050000918DF8E1
:1026F0000420B0E7197A237B994228BF1946C4E722
:10270000B0DF704766DF704710B50021044640888F
:10271000FFF7F8FF034608B9237210BD112801D155
:102720000123F9E76368BDE81040184760B159B16B
:102730000378DE2B0AD00B684360DE2303704FF66C
:10274000FF734380002070470E20704708207047B9
:1027500028B10378DE2B04D14180002070470E2081
:10276000704708207047F0B5054685B00C46F1B1BA
:10277000E8B10B78DE2B1AD182884B889A4204D1BB
:102780000B7A13B10846FFF7BFFF2B88112B32D00D
:10279000512B0ED0012B0AD12B7A012B07D1A988FE
:1027A0006288914203D123722046FFF7ADFF05B046
:1027B000F0BDAE886388B342F9D1AF79022FF6D16C
:1027C000AD7B2B1F022BF2D800211022684602F0AD
:1027D0006DFD052D14BF4FF4C073002369463046CC
:1027E0008DF80070ADF80430FFF78AFF0028DED0C6
:1027F00063689847DBE76388AA889A4204BF4FF66C
:10280000FF736380D3E7012804D0043805288CBF08
:102810000020012070474FF6FF73438000F082BA1A
:102820002DE9F041214E8AB000210822684631701E
:1028300002F03CFD4FF6FF7000F062FC4FF6FF78AF
:10284000044648F20967444513D0A4F58045ADB26B
:102850006A4602A92846FAF7B3FFB8420CD02846C8
:10286000FAF746FF48F20763984205460CD1012368
:1028700033700AB0BDE8F081204600F0E3FB20464B
:1028800000F03EFC0446DEE7002DF2D014220021C9
:102890000DEB020002F00AFD072305A88DF81430A5
:1028A000ADF818400795FFF7B6FFE2E75433002074
:1028B00070B5044686B014263246002101A802F005
:1028C000F5FCA0892378304D00F5804080B2042BC0
:1028D000ADF808003DD008D85A1E022A12D92B782C
:1028E0000BB1FFF79DFF06B070BD052BF7D16368F4
:1028F000002B44D113238DF804304FF6FF73ADF84D
:1029000008301DE043F6FE76B042E18904D901F5B6
:10291000804292B2B242E2D8DA1E534253418DF85D
:102920000D30A368049363688DF80C1063B9082315
:102930008DF804309DF8143043F001038DF8143005
:1029400001A8FFF768FFCAE709228DF80420059364
:10295000F6E743F6FE739842C1D8E389002BBED157
:1029600063683BB90A238DF8043000F06BFB012348
:102970002B70E5E70B228DF804200393F7E78DF821
:1029800004600393B9E700BF5433002073B50446D5
:102990000D46164600210822684602F087FCA5F580
:1029A0008041A4F580406B46324689B280B2FAF786
:1029B000EDFE002818BF052002B070BD30B51748E5
:1029C00089B0FAF719FD20BBFAF72CFD044610BBBD
:1029D00000F018FB0822214603A802F067FC03AAB6
:1029E00005A94CF20700FAF7DEFE10B1204609B047
:1029F00030BD01A905A8FAF725FE019B9D8805F5C4
:102A00008045ADB205A8FAF743FE284600F002FB68
:102A1000E5E70324EAE78624E8E700BFB1280200DF
:102A2000F0B5FF2887B004460E4615461F462BD842
:102A30000846FFF7E8FE38B303AA2046FFF7A6FFD3
:102A400018B10524204607B0F0BD01A903A8FAF784
:102A5000F9FD04460028F4D1019BAE705E8802990E
:102A60002E8027B9696003A8FAF712FEEAE73F68EB
:102A70006868B600B74228BF37463A4602F0EDFB19
:102A8000BE42F0D90C24DDE70724DBE70248082228
:102A9000002102F00BBC00BF4C330020F0B587B022
:102AA00006460F461546FFF7AEFE0446F8B1A6F5FA
:102AB0008040104A03A980B2FAF775FE18B10024CD
:102AC000204607B0F0BD01A903A8FAF7BBFD002816
:102AD000F5D1019BAE705A889B882A8003F580430C
:102AE000029A6A6003A83B80FAF7D2FDE8E7012466
:102AF000E6E700BF4C33002030B5FF2887B003461F
:102B00000C4615463BD889780846FFF77CFE00281E
:102B100035D0A3F58042ADF80020A1F58042ADF894
:102B200002206268019222880292184603AAFFF7E7
:102B30002DFF0528694603A80CD1FAF7CDFD48F210
:102B40000663984204461CD007D888B10324204667
:102B500007B030BDFAF7C4FDF1E748F207639842C9
:102B600011D048F20D63984214BF03241124EEE7FC
:102B7000002DECD0294603A8FAF72FFEE7E707243B
:102B8000E5E78624E3E71124E1E74FF6FF7000F064
:102B900041BAFF2808B505D800F042FAFFF740FE19
:102BA000002008BD0720FCE700F062BA00F08EBAF2
:102BB00000F0A6BA00F0AABA0A68084B70B50C2556
:102BC000032A01D9002006E005FB02F4E65A8642FA
:102BD00002D10A60181970BD0132F1E7AC3400204F
:102BE00037B500230D460446019301A9FFF7E4FF22
:102BF00038B18378AB4206D1837A9B0703D143680F
:102C00000BB903B030BD019B0133019301A92046EC
:102C1000ECE710B5044600F0CBFB204601F062FB68
:102C20002046FFF70BFA2046BDE81040FFF762B8D8
:102C300070B50E4E04460025237AAB420DD84FF6F0
:102C4000FF732380A370002363604FF47F432381CD
:102C5000A37A23F00303A37270BD617A2944C9B239
:102C6000304600F0FCFD0135E6E700BF9C34002053
:102C700013B50023CDE90033417A83788DF8023013
:102C80000446264800F0D2FD60B3237AA2788DF87E
:102C9000022003EB83039B00ADF80030531E01902C
:102CA000072B08D8DFE803F01607070707160418F4
:102CB0001423ADF800302246694632F8040BFFF7C2
:102CC0001BFF112815D00BD870B1072818BF03209F
:102CD00002B010BD0123ECE7838809339B08E8E7C5
:102CE000862811D00320F3E7A37A23F00303A3720D
:102CF000EEE7A37A23F0030343F00203A372084B29
:102D000001221A700020E3E7A37A23F0030343F0C3
:102D10000103A372024B01221A70D9E79C340020F0
:102D2000983400202DE9F047384EC16886B005463A
:102D3000324600233746506881421BD10C2000FBED
:102D400003702B78DFF8C880092B1AD0132B51D0D1
:102D5000082B51D16C7A002C4ED100284ED0FFF7B1
:102D600067FF2846FFF755FF98F800309BB906B07B
:102D7000BDE8F0870133042B02F10C02DBD1002007
:102D8000DFE76C7A002C37D1002837D0837A446093
:102D900043F002038372002588F800504FF00C09BD
:102DA0004FF0010A09FB05739B7A9907C3F34002B0
:102DB00001D4DB0724D588F800A002B904B330465B
:102DC000FFF756FFE0B14FF6FF73ADF806300C2366
:102DD0005D4386287B5BADF8083016BF0390062361
:102DE000072301A80CBF8DF804308DF80430FFF7DD
:102DF00010FFBCE70124B4E70024B2E70446B0E7C3
:102E00000135042D06F10C06CCD1B0E7AC3400201E
:102E100098340020154BF7B500221E464FF6FF757B
:102E20004FF0FF0C0C27104607FB02641D809D70BD
:102E300083F809C0A17A013221F00301042AA172AA
:102E400003F10C0303F8040C43F8080CECD15023F5
:102E5000CDE900230649074B07484FF4A07200F064
:102E6000D1FC002818BF032003B0F0BDAC34002013
:102E700058330020DC3400209C3400200023FFF76E
:102E8000CFBD00002DE9F04180460E4614461F4696
:102E9000002B4ED0CB1F012B4ED8531E032B4BD8EB
:102EA000FFF79EFE054610BBFF214FF6FF70FFF7B0
:102EB00097FE0546C8B1A0F8008086706B7AFF2B9C
:102EC0001AD11F48214600F0E2FCFF2868722DD17C
:102ED0004FF6FF732B8000236B604FF47F432B81F1
:102EE000AB7AA87023F00303AB72112022E0037ABF
:102EF000A342E3D00F201DE04FF00008697A10488C
:102F00002C7200F093FCC8B104EB84042401A4B239
:102F1000A408BE7078603C80B8F1000F04D0082E81
:102F200002D1A400063C8480002003E04FF0010899
:102F3000E4E70E20BDE8F0810720FBE70320F9E776
:102F40009C34002008B5FFF74BFE18B1FFF770FE68
:102F5000002008BD0520FCE713B5002304460193BB
:102F600001A9FFF729FE30B92046FFF712FE50B144
:102F7000072807D107E081782046FFF7E3FF20B15B
:102F8000052802D0032002B010BD019B013301933C
:102F900001A92046E5E7CB1F012B70B506460C467C
:102FA000154601D9072070BD1046FFF7FDFD00282A
:102FB000F8D021463046FFF713FE28B18470058013
:102FC000BDE87040FFF754BE0520ECE710B54FF6A2
:102FD000FF7304469C4208460AD14FF48071FAF709
:102FE0005BFD84B2B4F5807F09D14FF6FF7406E033
:102FF000FF2CFAD82146FAF72EFD0028F5D12046FD
:1030000010BD000002484022002102F04FB900BF6D
:10301000E03400200149FFF7D9BF00BFE0340020B1
:103020004FF6FF73984210B5044606D00449FFF7E7
:10303000CDFF231A5842584110BD0020FCE700BFC5
:1030400000350020FF2807B501460AD80190064840
:10305000FAF70FFD0199054803B05DF804EBFAF7A4
:1030600008BD03B05DF804FBE0340020003500200B
:10307000FF28014602D80248FAF705BD0020704734
:10308000E0340020FF28014602D80248FAF7FBBCD2
:1030900000207047003500204FF6FF73984270B54E
:1030A00018BF441C0E4614BFA4B20024A5B2FF2DC5
:1030B00002D94FF6FF7506E021463046FAF7E3FCE9
:1030C00001340028F2D0284670BD000070B50B49CD
:1030D0000A4EFFF7E1FF4FF6FF750446AC4201D1FF
:1030E000204670BD2046FFF7CDFF0028F8D02046CF
:1030F0003146FFF7D1FF0446F0E700BFE03400207F
:103100000149FFF7C9BF00BF0035002070B500249A
:10311000064E254621463046FAF7B5FC0134B4F593
:10312000807F0544F6D1284670BD00BFE034002002
:10313000F8B5074D074E074600243378A34200DC5C
:10314000F8BD55F8043B384698470134F5E700BF11
:103150002835002037350020074B1B7810B5044672
:103160004BB1FFF7AFF9204601F0F8F82046BDE873
:103170001040FEF781BE10BD3635002008B1FFF7C4
:10318000D7BF7047FFF7D4BFFFF7D2BFFFF7D0BF5D
:1031900008B5FFF713FC08B1032008BDFFF73AFE9E
:1031A0000028F9D101F0BEF80028F5D100F080FC2C
:1031B0000028F1D1FEF7E6FD0028EDD1FEF74AFF29
:1031C0000028E9D1054B4FF6FF721A80044B1860B6
:1031D000044B1870044B01221A70DEE734350020CE
:1031E0003C3500203835002036350020084B1B7850
:1031F00053B1084A1378022B08D8074941F8230035
:103200000133137000207047082070470420704776
:10321000363500203735002028350020034B1B7839
:103220000BB101F0B5B80820704700BF363500205B
:1032300008B5054B1B782BB101F0CAF8082808BF68
:10324000112008BD0820FCE73635002009B101F047
:10325000BDB87047034B1B780BB100F0A4BF08202A
:10326000704700BF36350020074B1B7810B50C4661
:103270002BB131B1FFF728F82080002010BD0820C5
:10328000FCE70E20FAE700BF36350020024B187825
:1032900008B1FFF78FBC704736350020034B1B7811
:1032A0000BB1FFF7ADB80820704700BF36350020DE
:1032B0002DE9F04F87B0814601932C4B1B7888464F
:1032C0001646002B50D04FF6FF70FFF76FFC00251D
:1032D0000423CDE9025302AB059304AA03AB0621F4
:1032E00004460495FFF79CFB072839D04FF6FF777B
:1032F000BB464FF0FF3AF0B1052825D04FF6FF73DB
:103300009C422FD1A34529D0A7420CBF0520002005
:10331000B9F1000F01D0A9F800B0B8F1000F01D049
:10332000C8F8005006B13780019B0BB1C3F800A06C
:1033300007B0BDE8F08F029BAB4224BFA3461D46F9
:1033400053453CBF27469A462046FFF72FFC03AB68
:1033500004AA06210446FFF763FBCCE70520D7E764
:103360000520E5E70320E3E70820E1E73635002004
:1033700038B50C4C0C4D00231A4621462846FFF761
:1033800097FF05280AD14FF6FF732B800023236097
:10339000431F58425841054B187038BD0028F7D1DB
:1033A0000120F8E720350020343500203835002092
:1033B000F0B5044687B08088FEF7B4FF23786080BC
:1033C000083B032B20D8DFE803F002213166637A43
:1033D0005BB93F4A116851B1E068814207D113607F
:1033E0003C4AA1881180E3600EE0012B0CD13A4BDE
:1033F0001B784BB1374BA2881B889A4204D1237AA1
:10340000062B01D1FFF7B4FF20465DE0637A002B65
:10341000FAD12F4A11680029F6D0E0688142F3D131
:103420002E4913600A68013A0A60DCE72C4F3B78AA
:1034300073B90125284B1B7833B1264BA2881B8812
:103440009A4201D1FFF794FF002DDDD107B0F0BD06
:103450004FF6FF70FFF7AAFB4FF6FF739842054641
:10346000E7D1FFF7A5FBA8420646E2D100251422CA
:10347000294601A83D7001F019FF0C2320468DF864
:103480000430ADF80860ADF80660FFF751FE01A802
:10349000FFF74EFECEE7124B1A78002AB4D0002177
:1034A000142201A8197001F001FF0D238DF80430DA
:1034B0004FF6FF73ADF80830ADF806302046A3682C
:1034C0000393FFF735FE01A8FFF732FEBEE700BF0A
:1034D0003C350020343500203835002020350020D0
:1034E000243500202DE9F041304B1B7888B006468A
:1034F000002B56D02E4B2F4C93E80300237801AFBE
:1035000087E8030043B12C4B1C68984654B1112442
:10351000204608B0BDE8F081FFF72AFF2378002B92
:10352000F5D0F0E7254A264D12882B68B2421DD10E
:10353000F3B11422214603A801F0B8FE0823304657
:103540008DF80C30FEF7EEFE0623ADF814309DF832
:103550001C30ADF80E0064F3000303A8ADF8106052
:1035600006948DF81C30FFF7E3FDD1E75A1C1AD002
:103570000133114A2B6039463046FFF7BDFA044645
:103580000028C5D00023C8F800302B68112803F1AB
:10359000FF332B60BBD08628BAD0072818BF03247E
:1035A000B6E70824B4E71324B2E700BF363500209D
:1035B00038550200383500203C35002034350020D5
:1035C0002035002076DF704713B5044669B901A99C
:1035D000FFF740FE43F20202904202D008B1F8F732
:1035E000FBFE9DF804309B070CD400212046FFF71A
:1035F0001FFE38B1112805D00D2805D11321204612
:10360000FFF7E0FF02B010BD0B28FBD043F202022F
:103610009042F7D0F8F7E0FEF4E7017811B940885E
:10362000FFF7D2BF072903D1806808B1F8F7D4BEED
:10363000704700002DE9F041037886B00446142B52
:103640003CD8DFE803F00B3B2D3B3B3B3E3B793B5B
:10365000793B3B3B3B3B3B3B3B7DA3008088FFF7FB
:1036600041FF862801D0112811D14F494F4A0B68DC
:10367000A08822F8130001335A4202F0070203F037
:10368000070358BF53420B6000F098F816E0132868
:1036900003D8474BC340DB0710D4F8F79DFE0DE07D
:1036A000037A012B0AD884881422002101A801F092
:1036B000FDFD01A8ADF80840FFF7BCFF06B0BDE86E
:1036C000F0813C4E3378002BF8D13B4D2B7843BB37
:1036D00001A8FAF78BF8044608B1F8F77DFEBDF8AB
:1036E0000A30002B14BF012200222A7017D101AA30
:1036F00019461846FFF7DCFD044648B9BDF804003A
:10370000FFF7CCFD044608B1F8F766FE01232B70E5
:10371000631F012B03D924B12046F8F75DFE002C6E
:10372000CCD1FAF70DF810B901233370C6E748F28F
:1037300007629042C2D0B0E71F4B01221A70BDE76A
:103740001C4B1A4D00241C701B4B1C70164B1F6821
:103750004FF6FF76E3195A4202F0070203F007031F
:1037600058BF534235F81380B0450BD014220021C6
:1037700001A825F8136001F099FD01A8ADF80880B3
:10378000FFF758FF0134082CE4D197E7094B0022DA
:103790001A70836848F20D6293423FF475AFB3F537
:1037A000064F8BD170E700BF44350020242700204E
:1037B000C100080040350020222700207FB51422D8
:1037C000002101A801F072FD062301A88DF8043044
:1037D000FFF730FF07B05DF804FB08B50378032B53
:1037E0000FD140881321FFF7EDFE43F20202904211
:1037F000034606D033F0080303D0BDE80840F8F7CD
:10380000EBBD08BD70B5DDE9045468B161B15BB1D1
:1038100004FB05F6964207D835B12CB1C0E9001378
:10382000C0E90254002070BD0720FCE738B50C4603
:10383000054608B9002038BD0368002BFAD040685F
:103840000028F7D0FF29F5D0BFF35F8FFAF71BF9F7
:103850000028EFD0E968286801FB0400EBE738B5E1
:103860000D46044690B1036883B1406870B1FF29EA
:103870000CD0BFF35F8FFAF706F938B16068BFF379
:103880005F8F2946BDE83840FAF7F3B838BD2DE917
:10389000F0418846064618B9FF242046BDE8F0816D
:1038A0000368002BF8D04368002BF5D00027FF24D5
:1038B000B368FDB2AB42EFD970682946FAF7CBF88E
:1038C000BFF35F8F40B9FF2C08BF2C462D1B01357D
:1038D0004545E2D00137EBE7FF2C07D1FF24F9E79C
:1038E00021463046FFF7BBFF0134E4B2AC42F7D3C8
:1038F000F4E77EDF70477FDF704786DF704710B5E3
:103900000378182B044602D1FDF7F8FF207010BD94
:1039100010B504464088FEF7D7FCA0802046BDE8DD
:10392000104000F0A5BC10B586B00446142200215A
:1039300001A801F0BBFC04230DEB03008DF804305B
:10394000ADF80640FFF7E4FF06B010BD30B587B014
:1039500005460C461422002101A801F0A7FC07230C
:1039600001A88DF80430ADF806500394FFF7D0FF9E
:1039700007B030BDF0B587B004460F4616460021AB
:10398000142201A81D4601F091FC03238DF8043098
:10399000094BADF8064019788DF80C7000222046CE
:1039A000ADF80E608DF81050FDF7CAFF01A8FFF7C3
:1039B000AFFF07B0F0BD00BF352700207FB5022361
:1039C0008DF804300388ADF8063043798DF80D107A
:1039D00013F0040F14BF0123022301A88DF80C304B
:1039E000FFF796FF07B05DF804FB000030B5114B00
:1039F0000A1E87B00C4618BF012219780546FDF74C
:103A00009FFF631E5A425A410B4B28461978FDF717
:103A100097FF1422002101A801F048FC012301A80E
:103A20008DF80430ADF806508DF80C40FFF770FFAC
:103A300007B030BD372700203627002073B501922C
:103A4000154A0D4611780446FDF762FF019B0146B9
:103A500000B3124A20461178FDF75AFF002804F5FA
:103A600080704FF0070180B214BF01260226FFF7D5
:103A700069FA019B014628B1052803D02046FFF7CB
:103A800065FF019B2A463146204602B0BDE87040E2
:103A9000FFF770BF2A46F7E73727002036270020B8
:103AA000024B0A781978FDF74BBF00BF342700207E
:103AB000F8B5104F104E114D114C3846FFF71FFF4F
:103AC0003046FFF71CFF2846FFF719FF2046FFF797
:103AD00016FF3B78182B0BD03378182B08D02B7897
:103AE000182B05D02378182B0CBF03200020F8BD1D
:103AF0000320FCE735270020372700203627002049
:103B0000342700202DE9F0418AB00E469046044645
:103B1000FDF7AAFE20220546002102A801F0C6FBFF
:103B2000012D08D1354B002219782046FDF708FFFA
:103B300036B9852715E0002D5AD143F2020052E034
:103B40002046FEF7C1FB4FF6FF73984210D10027C5
:103B50003378DB0720D42A4BCDF814800993012D4C
:103B600049D102AB324639462046FFF7C4FE3AE05F
:103B7000012DECD1214F20463978FDF7C9FE0028F0
:103B8000E5D12046FFF7CFFE39782046FDF7C0FE8D
:103B90000028DCD18527DBE7852FE0D004F5807095
:103BA0006B460122072180B2FFF76CF911281AD069
:103BB000E0B901465022019801F078FB01990B46CB
:103BC000204603F8345B029301F1180306934B1C63
:103BD000079311310A4BCDF814800993FEF786FB49
:103BE0000028BCD008200AB0BDE8F0810320FAE725
:103BF000002EA5D1852702AB0022B4E73427002090
:103C00004835002038B505460C46FDF72DFE012845
:103C100008D154B121462846FFF76BFE042808BF9F
:103C2000112038BD43F20200FBE72046F9E700000F
:103C30002DE9F0470388113B8AB00446092B74D85C
:103C4000DFE813F00A0073001F00480073007300E0
:103C500073007300A0003001037A84883D2BA74BCA
:103C60002046197841F23D0518BF4FF48855FDF7FD
:103C70004FFE002859D0002229462046FFF7DEFEDD
:103C800053E08088FDF7F0FD012802460FD1257A28
:103C90009A4BA0881978019005F00105C5F102053D
:103CA000EDB2FDF74DFE01982946FFF79FFE34F86F
:103CB000045F142200210DEB020001F0F7FA043436
:103CC00005238DF81430ADF81650079405A8FFF7BA
:103CD0001FFE2AE000F110063046FEF766FB4FF6A5
:103CE000FF7398420546A08822D1FEF7EDFA0546FB
:103CF000824BA088197801900122FDF721FE0198DE
:103D00000021FFF773FE4FF6FF739D4214D100258B
:103D100000232946A0881A46FFF7EFFD0828014630
:103D200003D010B3A088FFF711FE0AB0BDE8F087FA
:103D30002946FEF75BFBDBE705AA07212846FFF7CC
:103D40009DF80028E3D1A37ED907E0D5069D95F81C
:103D50004430DA0701D53435DAE7314605F146005B
:103D6000FEF70FFB0028F6D1D1E7A37EDB07DCD5F9
:103D7000002DDAD1A0882B4641F206022946FFF732
:103D8000F9FDD2E75D4B90F8088019788588B8F185
:103D9000000F79D1061D42462846FDF7D1FD617A14
:103DA00011F0040103D13046FFF708FEBDE705F529
:103DB00080791FFA89F903AB012207214846FFF7F2
:103DC00061F8074628B101462846FFF7BFFD414686
:103DD000E9E72846FEF778FA4FF6FF739842044663
:103DE00082462FD101460498FEF750FA504504460A
:103DF000804678D0DFF80CA101462846FEF7F6FA97
:103E00009AF800102846FDF783FD8046D0B9284671
:103E1000FFF789FD9AF800102846FDF779FD014665
:103E20000028C0D0072122464846FFF7B4F80146D3
:103E300050B90121B7E721462846FEF7D7FA4FF0DF
:103E40000108EFE7B846EDE786280ED114220021DD
:103E50000DEB020001F02AFA062305A88DF81430B4
:103E6000ADF81650FFF754FDE3E72846FFF76EFD67
:103E700000213046FFF7A2FDB8F1000F3FF455AF27
:103E80002046FEF7BDFA50E7427A284602F00302C8
:103E90000192FDF73DFD019A00283FF446AF4146EF
:103EA0002846EBE6164B80881978FDF731FD05466C
:103EB00000287FF43AAFA088FDF7EAFC0146A0880D
:103EC00019B9012341F2060259E70C4B2A46197829
:103ED000FDF736FD02238DF81430A388ADF81630B7
:103EE000ADF81C50F2E6FEF750FE40450446A2D164
:103EF00004212846FFF72AFD394654E735270020DC
:103F0000372700203427002058B3027802F08203BC
:103F1000802B25D0C2F30213042B21D802F0F20328
:103F2000322B1DD041788378994219D8062917D9A8
:103F3000102B15D8C17811F0040311D10079430773
:103F40000ED4084301070BD4D30700F0030003D4B9
:103F5000B0FA80F040097047003818BF0120704760
:103F60000020704770B515460E4614220021044605
:103F700001F09CF92846FEF7A7F92670A08065801D
:103F8000204670BDFFF7FAB810B50378182B044629
:103F900002D1FDF7B3FC207010BD30B531F008033D
:103FA00087B00C4615461BD0112919D00D290246A1
:103FB0001AD1032101A8FFF7D5FF9DB12B7803F09B
:103FC0000103C3F10203DBB28DF80C3000238DF83E
:103FD000103041F20113ADF80E3001A8FFF7D2FF07
:103FE00007B030BD0223EFE7072101A8FFF7BAFFB2
:103FF0000394F2E72DE9F043064689B01746984648
:104000000D4609BB334BCDE904111B68039303AC88
:1040100094E80700E94689E8070032460521204672
:10402000FFF7A0FF2046CDE90559FFF7ABFF2A4B6C
:10403000DDF800901B784BB99DF8093033B90525A0
:10404000284609B0BDE8F0834FF000093A464946DA
:104050003046FFF7D7FDA0F111035A425A411F4BDA
:10406000044619783046FDF76BFC112C1BD8072C41
:104070000CD8002C0CBF00250325B8F1000FDFD0B1
:104080004A4621463046FFF788FFD9E7A4F10803E6
:10409000092B06D8DFE803F01B05051B051B0505EA
:1040A000050D0325E9E743F20205AC4218BF0325DD
:1040B000E3E70B4B2A4619783046FDF741FC094BE4
:1040C0003A4619783046FDF73BFC0025D5E72546F2
:1040D000D3E700BF94350020913500203A27002017
:1040E000392700203827002013B50A4B19780446D9
:1040F000FDF70EFC084B019019782046FDF708FCEF
:10410000019A01460123204602B0BDE81040FFF7A6
:1041100071BF00BF38270020392700202DE9F0416A
:104120001B4B88B00027CDE904771B68039303ADD0
:104130000446884695E807006E4686E80700224652
:1041400005212846FFF70EFF2846CDE90586FFF733
:1041500019FF104B00991A682046FFF7D3FCA0F115
:1041600011035A425A410C4B054619782046FDF777
:10417000E7FB0A4B3A4619782046FDF7E1FB009A27
:1041800029462046FFF709FF08B0BDE8F08100BFCF
:1041900094350020883500203B2700203A27002056
:1041A0000021FFF7BBBFF7B507460C46002945D0F5
:1041B000FDF75CFB0546002842D03846FEF784F840
:1041C00006464FF6FF70301AA5F1020318BF012012
:1041D0005D425D41237845EAC00523F009031D4394
:1041E00025703846FDF754FB237860F341032370B4
:1041F0003846FDF75FFB237860F38203237038466F
:10420000FDF76AFB0546B8B93846FDF741FB50B1EA
:104210006A4607213046FEF731FE58B9019B93F8F4
:10422000440000F00100237860F3041323700020A1
:1042300003B0F0BD2846F6E70120F4E70E20F7E7CB
:1042400043F20200F4E713B5E0230C4601A98DF810
:104250000430FFF7A8FF9DF80420237828B9934382
:104260000CBF0120002002B010BD0020FBE70000C1
:1042700013B50378052B044605D0122B09D0204630
:10428000FFF780FE03E081684088FFF747FF02B038
:1042900010BD134B1A68FAB14088FDF7F9FA0146D0
:1042A000E0B1227A6088C2F34003C2F300019B00B0
:1042B000C2F3800243EAC10343EA021301A98DF865
:1042C0000430FFF7C0FF80F00100C2B20021608817
:1042D0000123FFF78FFED2E70121F8E70246F6E758
:1042E0009435002008B503780B2B0FD8072B0FD976
:1042F000084B094918780022FDF73CFB074B084999
:1043000018780022BDE80840FDF734BB132BEFD02E
:1043100008BD00BF3B270020A14102003A27002032
:10432000E940020010B50948094CFFF72DFE094885
:10433000FFF72AFE0848FFF727FE2046FFF724FE76
:104340002378182B0CBF0320002010BD3A27002033
:104350003B270020382700203927002008B5FFF729
:1043600067FC074B074918780022FDF703FB064B53
:10437000064918780022BDE80840FDF7FBBA00BFE7
:104380003B270020A14102003A270020E94002001B
:1043900010B5044630B90A4B18600A4B01221A7056
:1043A000002010BDFFF7B0FD38B1074B22681A603E
:1043B00022791A71024A1360EFE70720F1E700BF84
:1043C00094350020913500208C350020FFF768BB24
:1043D00000230A461946FFF70DBE10DF704711DFB4
:1043E0007047000013B5044609496846F9F774FEA2
:1043F000019808B902B010BDD0E9002120469047CD
:1044000018B16846F9F772FEF2E71120F2E700BF33
:104410004455020013B5044607496846F9F75CFEA7
:10442000019B0BB902B010BD2046D3E90021904793
:104430006846F9F75BFEF3E75C550200064B9A68A5
:1044400022B11A6822F480021A607047034B4FF4BD
:104450008002C3F880207047C427002000E100E0FC
:104460000B4991F816335A09EC231341DB0706D5A3
:10447000084B9A683AB94FF480030B60704742F2D8
:104480000200F7F7A9BF1A6842F480021A60704769
:1044900000E100E0C4270020F7B5194F3C7864BB69
:1044A000184E012520463570FFF79CFF112821D0BA
:1044B0002046FFF7AFFF144B8DF8034018680190BA
:1044C0000DF10300F8F75EF9104901A8FFF785FF29
:1044D0000446B0FA80F0400938709DF80300F8F700
:1044E00075F93CB90A4B34701C70FFF7B9FF2846C8
:1044F000FFF790FF204603B0F0BD0824FAE700BFA5
:10450000993500209835002040550200F5C3010080
:104510009A350020F7B5154F3B781BB3144E012098
:104520003070FFF75FFF11284FF000051CD002200C
:10453000FFF770FF0DF107008DF80750F8F722F92B
:10454000FFF74DFF04469DF807003D70F8F73EF970
:104550002CB93470FFF772FF0320FFF75BFF204692
:1045600003B0F0BD0824FAE72C46F8E7993500209F
:1045700098350020054B1B7833B1054B1B780BB1E8
:10458000FFF7C8BFFFF788BF0820704798350020A5
:1045900099350020014B1878704700BF99350020ED
:1045A00007B508496846F9F797FD019B13B903B0B1
:1045B0005DF804FBD3E9002090476846F9F796FDC3
:1045C000F3E700BF50550200FFF7EABF60DF704716
:1045D00069DF704761DF704730B5114B1B7891B0D0
:1045E000E3B1104D34240DF1020103A8ADF80240EF
:1045F000FFF7F0FF70B9294601A8F9F76DFD029B9E
:10460000002BF0D003A8D3E90021904701A8F9F7C7
:104610006DFDF4E7052801D0F7F7DEFE11B030BDDF
:104620009B3500206855020030B5054685B00C4624
:1046300000294AD0264B0B600C22002101A800F073
:1046400035FE062322688DF8045001A9012520209B
:10465000ADF808308DF80650FFF7BAFF0C220021A4
:1046600001A800F023FE22688DF8055001A9402022
:10467000FFF7AEFF0C22002101A800F017FE226810
:104680008DF8045001A92846FFF7A2FF0C22002153
:1046900001A800F00BFE4FF4B0632268019301A95A
:1046A000A120FFF795FF0C22002101A800F0FEFDDC
:1046B0009DF8043022682B4301A9A0208DF8043016
:1046C000FFF786FF002005B030BD0E20FBE700BFDE
:1046D0000C26002008B5FFF779FF10B9014B012225
:1046E0001A7008BD9B3500204BDF70471FB50D4C7D
:1046F00001A8FFF7F9FF70B9214602A8F9F7ECFC11
:10470000039B002BF4D00198D3E90021904702A825
:10471000F9F7ECFCF4E7052801D0F7F75DFE04B0EB
:1047200010BD00BF7455020030B591EA030F00F1CF
:104730008480841A71EB030C05D2121953EB0C031D
:10474000001B71EB0C0140F2000CCFF6E07C1CEA80
:10475000430F54D0BCEB410F61D90C0DA4EB135E99
:1047600031EA0C0141F4801133EA0C0343F4801365
:10477000DEF1200C2AD303FA0CF5401941F10001B7
:1047800022FA0EF5401923FA0EF5694112FA0CF2DD
:10479000CD0208D349085FEA30005FEA320228BF41
:1047A00042F001020134013C5FEA500C72F1004218
:1047B00050F1000051EB04514FF4001313EB410F83
:1047C00038BF30BD090D0905002030BDBEF1200EF7
:1047D000BEF1200F1ED223FA0EF5401941F100015F
:1047E000CEF1200C124218BF012203FA0CF52A4325
:1047F000CEE711EA5C0F04BF0020002130BD1CEAA7
:10480000410F04BF01F00041002030BD01F0004124
:10481000002030BD21F4801101EB045130BD004275
:1048200018BF41F00101BCEB410F08BF30BD4FF094
:10483000FE4141F47801002030BD83F00043841A2A
:1048400071EB030E07D28EF0004E001B71EB0E01D0
:10485000121953EB0E0340F2000CCFF6E07C1CEA79
:10486000430FC6D0BCEB410F72D90C0DA4EB135E05
:10487000C90241EA5051C00241F00041DB0243EA63
:104880005253D20243F00043DEF1200C41D312FA1E
:104890000CF522FA0EF203FA0CF542EA050218BFF3
:1048A00042F0010223FA0EF3801A9941E30AC4F39D
:1048B0000A0411F0404F03D418D0013C4000494194
:1048C000013C23D44205C00A40EA4150C90A51EADA
:1048D000C3715FEA500C72F1004250F1000051EBDD
:1048E000045130BD01002FD00020203C0029F9D018
:1048F000B1FA81FCDCF1200E11FA0CF130FA0EF560
:1049000010FA0CF02943A4EB0C04D9E70020D907D6
:1049100030BDAEF1200EBEF1200F0DD2CEF1200C35
:1049200003FA0CF533FA0EF32A4318BF43F00103E0
:10493000C01A61F10001B9E721F00041C00A40EA64
:104940004150C90A01EB045130BD0020002130BDA7
:10495000004218BF41F00101BCEB410F7FF467AF8B
:10496000BCEB430F3FF463AF30BD00BF83F00043A7
:10497000FFF7DABEF0B540F2FF7681EA030C16EAE3
:10498000115E1EBFB64516EA1355B5425AD021EA4C
:10499000465141F48011A1FB024723EA465343F4F8
:1049A0008013AE44A0FB03650CF0004C36197D412A
:1049B000A1FB034747F10003A0FB0217F61965416D
:1049C00053F10003094218BF46F0010640F2FE749D
:1049D000B3F5007F13D2AEF5806EA6452BD24CEA1C
:1049E0000331280341EA155140EA165032034508C5
:1049F00072F1004250F1000051EB0E51F0BDAEF2E9
:104A0000FF3EA64517D24CEAC321E80241EA5551C0
:104A100040EA5650F202450872F1004250F100009F
:104A200051EB0E51F0BD0CF0004141F0FE4141F45C
:104A300070010020F0BD1EEA0E0FF4D50CF000410D
:104A40000020F0BD16EA115F04BF01F00041002014
:104A5000004218BF41F0010116EA135F04BF03F0E2
:104A600000430022124218BF43F0010306EA135428
:104A7000B44218BF9EEA060F03D00CF0004100209C
:104A8000F0BD21F0004123F00043B1EB065F06D8F2
:104A9000B3EB065F03D8002918BF002BC3D140F247
:104AA0000001C7F6F8710020F0BD00BF2DE9F0430A
:104AB00091EA030E0EF0004E40F20007CFF6E077C9
:104AC00017EA41051EBF95EA070F17EA430595EA65
:104AD000070F00F0A1807F0D17EA135623EA475312
:104AE00043F4801317EA115521EA475141F480112C
:104AF000AD1B05F2FD354FEAD31C1CF1010C4FF044
:104B00000047B7FBFCF77F01A2FB079C0024E3FBF7
:104B100007C4DCF1000CD9F100097CF1000CA0FB0A
:104B200007620020E1FB072000275FEAC628E0FBC0
:104B30000987760D46EAC226520DF61900277A41FA
:104B4000E0FB0C625FEAC823E2FB09375FEA5858D2
:104B500048EAC628760D18EB070800214E41E2FB13
:104B60000C8602EBC020DA02E6FB09215B0D43EA6A
:104B7000C8235FEA58585B18002758EB0708E6FB84
:104B80000C38D102E8FB0917520D42EAC3225B0D33
:104B9000D21900277B41E8FB0C2308EBC6265FEA0D
:104BA000C128E3FB0987490D41EAC221520DC91909
:104BB00042F10002E3FB0C12470019EB08095CEB21
:104BC000010C72EB040453EBC62047EB565300264E
:104BD000B3F5000F7641AD190236D6F1200910FA6F
:104BE00009F4F04013FA09F21043F340E40F0019FE
:104BF00043F10003B3F5001F24BF5B08013540F209
:104C0000FE77BD4204D24EEA05511944BDE8F08357
:104C10002D4224D5714626E0004218BF41F0010123
:104C2000124218BF43F00103B7EB410F2CBFB7EBA3
:104C3000430F1BE0B7EB410F04BFB7EB430F15E089
:104C400017EA410F04BF17EA430F0FE017EA410FBD
:104C5000E0D017EA430F02D0B7EB430FDAD04EF0A3
:104C6000FE4141F470010020BDE8F08340F20001F4
:104C7000C7F6F871F7E700BF4FF4001C1CEB410FBB
:104C800098BF1CEB430F0CD850EA410C08BF52EA06
:104C9000430C08D0904208BF99420CBF012000206D
:104CA0007047002070470120704700BF4FF4001C80
:104CB0001CEB410F98BF1CEB430F11D851EA030CBA
:104CC00050EA4C0C5CEA020C0AD004D282428B41BE
:104CD0008041404270479042994180414042704734
:104CE000002070474FF4001C1CEB410F98BF1CEBD9
:104CF000430F11D851EA030C50EA4C0C5CEA020C49
:104D00000AD004D290429941804140427047824289
:104D10008B41804140427047002070470B0D40F2AC
:104D20001E42D21A09DBCB0243EA505040F0004049
:104D3000202A28BF2022D0407047490060EB0000A5
:104D4000704700BF80B110F0004248BFD0F10000B2
:104D5000120D02F21D42B0FA80F18840521AC30AC5
:104D6000400503EB025170470100704750B140F21B
:104D70001D42B0FA80F18840521AC30A400503EB85
:104D80000251704701007047C0F3C75191B1420012
:104D90004FEA40704FEAD2014FEA310101F1605110
:104DA000B2F17F4F38BF704701F1605118BF41F435
:104DB0000021704710F000410020704701F00042D0
:104DC0008B1AA3F16051B1F5801F0ADBB1F17F6F3F
:104DD00009D242EAC102C10071F1004142EB5070B8
:104DE00070471046704701285B4113F5001F04D837
:104DF00042F0FE4040F400007047C90041EA5070A4
:104E000040EA020040F4800040F08040704700BF5C
:104E100051EC100B0128494111F5001F8CBF0120F6
:104E20000020704770B555EC104B0646002210EE7E
:104E3000100A00232946FFF71FFF20B1002345EC8D
:104E4000104B336070BD25F0FF4121F4E00141F0CB
:104E50007F53C5F30A51224643F40013A1F2FE31F9
:104E600043EC102B316070BD2DE9704355EC104BB5
:104E70000646002210EE100A00232946FFF7FCFE2A
:104E8000B8B9C5F30A53334440F2FE72934214DCBE
:104E9000002EA04601DB002B0FDB002B09DD25F0E7
:104EA000FF4222F4E00242EA035949EC108BBDE8CC
:104EB00070839FED070BBDE8708300F091F9084BFC
:104EC0001B6803609FED040BBDE87083AFF30080A7
:104ED0000000000000000000000000000000F07F63
:104EE00080550200000000002DE9F04F85B055EC20
:104EF000104BFFF78DFF002840F0C18000220023F7
:104F000020462946FFF7B8FE002840F0BD80002269
:104F1000002320462946FFF7E5FE002840F0AF8039
:104F200045EC104B03A8FFF77DFF55EC104B76A323
:104F3000D3E9002310EE100A2946FFF7B7FE002838
:104F400040F0A780039B204629465C1E00226C4B44
:104F50000394FFF70BFD04460D4645EC104B4FF054
:104F6000FF30FFF781FF664B51EC100B0022FFF77B
:104F7000DBFB02460B4620462946FFF797FD02461B
:104F80000B4606460F46FFF7F5FC49A3D3E900237D
:104F900004460D46FFF7EEFC47A3D3E90023FFF7D5
:104FA000C3FB47A3D3E90023804689462046294610
:104FB000FFF7DCFC22462B46FFF7DCFC42A3D3E9DB
:104FC0000023FFF7B1FB424682468B464B46204604
:104FD0002946FFF7CFFC3EA3D3E90023FFF7C6FC29
:104FE0005246804689465B4620462946FFF7C2FC6A
:104FF00039A3D3E90023FFF7B9FC02460B4640462C
:105000004946FFF753FD02460B4620462946FFF767
:10501000B1FC32463B46FFF7ADFC02460B46039817
:10502000CDE90023FFF78EFEDDE9002304460D469F
:1050300030463946FFF778FB29A3D3E9002306461B
:105040000F4620462946FFF795FC02460B463046A0
:105050003946FFF769FB24A3D3E9002306460F4630
:1050600020462946FFF786FC02460B463046394665
:10507000FFF75AFB41EC100B05B0BDE8F08F9FED38
:105080001C0B05B0BDE8F08F9FED1B0B05B0BDE814
:10509000F08F0022204629461A4BFFF767FC024694
:1050A00045EC104B4FF0FF3014460D4659E700BF5A
:1050B00029BD56B31544E9BFEDAF16204A62304012
:1050C0000FCE674B80D541407E2615FA8380734012
:1050D0009AB5B312FF07504077900D9CFE0B8840A5
:1050E000A80C615C10D02BBF000000000030E63F30
:1050F000000000000000F87F000000000000F0FF4A
:105100000000E03F0000F03FCD3B7F669EA0E63F01
:1051100053EA020C61D02DE9F04BB3FA83F51E007F
:1051200007BFB2FA82F502FA05F403FA05F416464F
:10513000C5F120051EBF22FA05F73C43203556EA8B
:10514000044C4FEA144418BF0134A3464FF0000941
:10515000C846904271EB030C39D3094207BFB0FA3D
:1051600080F700FA07F6B1FA81F701FA07F6C7F1FE
:1051700020071EBF20FA07FC46EA0C062037B6FBC4
:10518000FBFC7F1B103F07F01F04C4F120060CFA44
:1051900004F42CFA06F644BF34460026202FA4BFA0
:1051A0002646002454EA060C08BF012418EB040824
:1051B00049EB0609A4FB027CC01B06FB02CC04FBE6
:1051C00003CC71EB0C01904271EB030CC5D20B4682
:1051D000024649464046BDE8F08BB2FBF3F20000C0
:1051E00000B5F7F7F5F8024B18445DF804FB00BF73
:1051F000080000007AB370B414460F2A15D902468D
:105200000B4640EA010515F0030F01D0013C0EE00A
:10521000194610460432043306680D68AE4204D1C4
:1052200010461946043C042CF2D8013C0ED00A4624
:1052300003460444114618460133013206780D78BE
:10524000AE4203D118461146A342F3D100780B7841
:10525000C01A70BC704700207047844640EA0103C2
:1052600013F0030F18D18446202A0BD32DE9F00741
:10527000B1E8F807A0E8F807A2F12002202AF7D247
:10528000BDE8F007042A07D351F8043B40F8043B7B
:10529000A2F10402042AF7D2002A05D011F8013B3A
:1052A00000F8013B013AF9D1604670478446002A74
:1052B0002DD010F0030F04D000F8011B013A26D0C6
:1052C000F7E7C9B241EA012141EA0141202A12D39C
:1052D000A2F120022DE9F0030B460C460D460E46C6
:1052E0000F4688468946A0E8FA03203AFBD2BDE87B
:1052F000F00320320BD0042A05D340F8041B043AF3
:1053000005D0042AF9D200F8011B013AFBD160460E
:10531000704700F1010110F0030F11D010F8012BBC
:10532000002A23D010F0030F0AD010F8012B002A16
:105330001CD010F0030F03D010F8012B002A15D059
:105340002DE970004FF001324FF0803350F8044BDC
:10535000A4EB020525EA04051D4000D1F6E7A0F103
:10536000040070BC10F8012B002AFBD1A0EB010057
:02537000704784
:10537400F5DD01000000000001E50100000000006F
:10538400511702000000000009140200702B0020D5
:10539400E9250200A82F002091150200000000005A
:1053A4005931020000000000A5020200CC2F0020A9
:1053B40067270200C02F00208DF3010000000000C9
:1053C4009DDE010000000000E9E50100000000008E
:1053D400D945020000000000ED4602000000000074
:0853E400D5DC0100000000000F
:1053EC000000000000000000DDD201000000000001
:0453FC0000000000AD
:1054000001000600000000003C27002029C4010024
:105410000338FDD8704700000000FFFFDEC0ADDE9E
:10542000FE011EF1DEC0ADDEFF011EF10010000026
:10543000040000000100000019DD0100F9DC01009A
:10544000E9DC010029DF0100DDDE0100BBDC010039
:10545000BFDC0100C5DC0100002A0020C4530200AB
:10546000C4530200040000004B696E6574726F6ED5
:1054700020536D6172742053686F7765720031320A
:105480003334353600000000000000000200000246
:1054900000000000064100000100020201010000BE
:1054A00001000000D007000006000000002B0020D3
:1054B0000338FDD870470000302B0020502B00200F
:1054C00020300020010001006030002003000000B7
:1054D00040300020004002402400040078300020CA
:1054E000A03000208DAAC011A0AAF5B0F2402FE193
:1054F000000022E61E1E1E1E0000001E0000001EF0
:105500001E05000000000000183100203831002086
:10551000583100200100FFFF0000000001000000E2
:105520000100010030550200010001003455020065
:1055300001000000000000000100060020350020EE
:1055400000100201E4530200EC53020008000000C6
:10555000D4530200E453020008000000C4530200C8
:10556000D45302000800000084530200C453020018
:105570000800000074530200845302000800000079
:045580002200000005
:1055840000100140110004000090D0030014020038
:10559400FFFFFFFF417665726167652053686F778F
:1055A40065722057617465722054656D706572610F
:1055B400747572650A556E69743A206343656C7339
:1055C400697573005265616C2054696D652057617B
:1055D4007465722054656D70657261747572650AC4
:1055E400556E69743A206343656C7369757300433F
:1055F400757272656E742053686F77657220447596
:10560400726174696F6E2E0A556E69743A2053651F
:10561400636F6E64730043757272656E74205368B1
:105624006F77657220494400546F74616C20576130
:1056340074657220636F6E73756D7074696F6E2E0E
:105644000A556E69743A206D696C6C696C69747280
:10565400650043757272656E742053686F77657266
:1056640020576174657220466C6F772E0A556E69F7
:10567400743A206D696C6C696C697472652F73651A
:1056840063000100FFFFFFFFFFFFFFFFFFFFFFFFBE
:0C569400FFFFFFFF18181818181818184E
:040000031000C375B1
:00000001FF
